:020000040800F2
:100000006F00C015000000000000000000000000AC
:1000100000000000000000000000000000000000E0
:1000200000000000000000000000000000000000D0
:1000300000000000000000000000000000000000C0
:1000400000000000000000000000000000000000B0
:1000500000000000000000000000000000000000A0
:1000600000000000485900080000000000000000E7
:100070000000000000000000000000000000000080
:100080000000000000000000000000000000000070
:100090000000000000000000000000000000000060
:1000A0000000000000000000000000000000000050
:1000B0000000000000000000000000000000000040
:1000C000A05900080000000000000000000000002F
:1000D0000000000000000000000000000000000020
:1000E0000000000000000000000000000000000010
:1000F000000000004C590008000000000000000053
:1001000000000000000000000000000000000000EF
:1001100000000000000000000000000000000000DF
:1001200000000000000000000000000000000000CF
:1001300000000000000000000000000000000000BF
:1001400000000000000000000000000000000000AF
:1001500000000000000000002859000873700430FF
:10016000170500001305C5FF930510009395D501F1
:10017000637EB50093D52500637AB50017050000AE
:10018000130505013305B500670005009302002043
:1001900073A0027D970200009382C2E673907230D2
:1001A00097A20000938202727390C27E73E0C07EB9
:1001B00097A2000093820261739052309711001849
:1001C0009381C1CA178100181301C1E317D500003C
:1001D000130585C8970500189385C5E21706001812
:1001E0001306C64A63FCC5008322050023A0550000
:1001F0001305450093854500E3E8C5FE1705001883
:100200001305C548938581786378B50023200500E0
:1002100013054500E36CB5FE73F00232EF20400693
:100220001305000093050000EFA000556F000000CB
:1002300073E002326780000073F0023267800000D2
:100240000000000000000000010203040607080986
:100250000000000001000000020000000300000098
:10026000EC4900086C5000088C490008984F0008C1
:100270008C490008F84E00087C4B00080C4D000823
:10028000144D0008844D0008684E0008B04E000868
:10029000F04E000894490008A8490008D049000819
:1002A000160347006900670061004400650076009E
:1002B0006900630065000000380347004400330014
:1002C000320020005500530042002000430044004B
:1002D00043002000410043004D00200069006E00F3
:1002E00020004600530020004D006F0064006500B0
:1002F000000000002E034700440033003200580085
:10030000580058002D0033002E0030002E00300021
:100310002D0037007A003800780039007900650038
:10032000720000001201000202000040E9288A0168
:10033000000101020301000050CE0008A0020008E5
:10034000B8020008F4020008C8610008E46100086F
:10035000F86100081C6200083C6200086062000846
:100360007462000898620008AC620008D06200085D
:10037000F4620008186300082C630008506300084A
:1003800064630008886300083C3F786D6C207665E4
:100390007273696F6E3D22312E30223F3E3C214404
:1003A0004F43545950452074617267657420535906
:1003B0005354454D20226764622D746172676574E1
:1003C0002E647464223E3C746172676574207665A5
:1003D0007273696F6E3D22312E30223E3C6665613C
:1003E00074757265206E616D653D226F72672E6750
:1003F0006E752E6764622E72697363762E637075F4
:10040000223E3C726567206E616D653D227A6572A1
:100410006F222062697473697A653D22333222202B
:100420007265676E756D3D22302220736176652D91
:10043000726573746F72653D2279657322207479D9
:1004400070653D22696E74222067726F75703D225F
:1004500067656E6572616C222F3E3C726567206E27
:10046000616D653D227261222062697473697A65EB
:100470003D22333222207265676E756D3D22312236
:1004800020736176652D726573746F72653D227994
:1004900065732220747970653D22696E742220672D
:1004A000726F75703D2267656E6572616C222F3EBA
:1004B0003C726567206E616D653D2273702220621B
:1004C000697473697A653D22333222207265676EE2
:1004D000756D3D22322220736176652D72657374CD
:1004E0006F72653D227965732220747970653D22B3
:1004F000696E74222067726F75703D2267656E6544
:1005000072616C222F3E3C726567206E616D653DA5
:10051000226770222062697473697A653D223332E2
:1005200022207265676E756D3D22332220736176DD
:10053000652D726573746F72653D22796573222033
:10054000747970653D22696E74222067726F7570D0
:100550003D2267656E6572616C222F3E3C72656755
:10056000206E616D653D227470222062697473692A
:100570007A653D22333222207265676E756D3D22A9
:10058000342220736176652D726573746F72653DD8
:10059000227965732220747970653D22696E742218
:1005A0002067726F75703D2267656E6572616C229F
:1005B0002F3E3C726567206E616D653D227430226E
:1005C0002062697473697A653D2233322220726534
:1005D000676E756D3D22352220736176652D7265DB
:1005E00073746F72653D227965732220747970652A
:1005F0003D22696E74222067726F75703D226765B7
:100600006E6572616C222F3E3C726567206E616D73
:10061000653D227431222062697473697A653D22D6
:10062000333222207265676E756D3D22362220734B
:100630006176652D726573746F72653D227965739D
:100640002220747970653D22696E74222067726F72
:1006500075703D2267656E6572616C222F3E3C723B
:100660006567206E616D653D227432222062697477
:1006700073697A653D22333222207265676E756D2B
:100680003D22372220736176652D726573746F7217
:10069000653D227965732220747970653D22696E0B
:1006A00074222067726F75703D2267656E65726196
:1006B0006C222F3E3C726567206E616D653D22663F
:1006C00070222062697473697A653D223332222078
:1006D0007265676E756D3D22382220736176652DD7
:1006E000726573746F72653D227965732220747927
:1006F00070653D22696E74222067726F75703D22AD
:1007000067656E6572616C222F3E3C726567206E74
:10071000616D653D227331222062697473697A6567
:100720003D22333222207265676E756D3D2239227B
:1007300020736176652D726573746F72653D2279E1
:1007400065732220747970653D22696E742220677A
:10075000726F75703D2267656E6572616C222F3E07
:100760003C726567206E616D653D226130222062BA
:10077000697473697A653D22333222207265676E2F
:10078000756D3D2231302220736176652D7265735F
:10079000746F72653D227965732220747970653DAE
:1007A00022696E74222067726F75703D2267656ED4
:1007B0006572616C222F3E3C726567206E616D65CB
:1007C0003D226131222062697473697A653D22336A
:1007D0003222207265676E756D3D223131222073A1
:1007E0006176652D726573746F72653D22796573EC
:1007F0002220747970653D22696E74222067726FC1
:1008000075703D2267656E6572616C222F3E3C7289
:100810006567206E616D653D2261322220626974D8
:1008200073697A653D22333222207265676E756D79
:100830003D2231322220736176652D726573746FAB
:1008400072653D227965732220747970653D226955
:100850006E74222067726F75703D2267656E6572D7
:10086000616C222F3E3C726567206E616D653D2292
:100870006133222062697473697A653D22333222C2
:10088000207265676E756D3D22313322207361766B
:10089000652D726573746F72653D227965732220D0
:1008A000747970653D22696E74222067726F75706D
:1008B0003D2267656E6572616C222F3E3C726567F2
:1008C000206E616D653D2261342220626974736916
:1008D0007A653D22333222207265676E756D3D2246
:1008E00031342220736176652D726573746F726581
:1008F0003D227965732220747970653D22696E749A
:10090000222067726F75703D2267656E6572616C3B
:10091000222F3E3C726567206E616D653D22613518
:10092000222062697473697A653D22333222207213
:1009300065676E756D3D2231352220736176652DB8
:10094000726573746F72653D2279657322207479C4
:1009500070653D22696E74222067726F75703D224A
:1009600067656E6572616C222F3E3C726567206E12
:10097000616D653D226136222062697473697A6512
:100980003D22333222207265676E756D3D2231360D
:100990002220736176652D726573746F72653D22D6
:1009A0007965732220747970653D22696E74222006
:1009B00067726F75703D2267656E6572616C222F7C
:1009C0003E3C726567206E616D653D226137222075
:1009D00062697473697A653D2233322220726567D9
:1009E0006E756D3D2231372220736176652D7265FB
:1009F00073746F72653D2279657322207479706516
:100A00003D22696E74222067726F75703D226765A2
:100A10006E6572616C222F3E3C726567206E616D5F
:100A2000653D227332222062697473697A653D22C2
:100A3000333222207265676E756D3D223138222077
:100A4000736176652D726573746F72653D22796589
:100A5000732220747970653D22696E74222067725A
:100A60006F75703D2267656E6572616C222F3E3C2A
:100A7000726567206E616D653D2273332220626965
:100A80007473697A653D22333222207265676E7510
:100A90006D3D2231392220736176652D7265737444
:100AA0006F72653D227965732220747970653D22ED
:100AB000696E74222067726F75703D2267656E657E
:100AC00072616C222F3E3C726567206E616D653DE0
:100AD000227334222062697473697A653D2233324D
:100AE00022207265676E756D3D223230222073615F
:100AF00076652D726573746F72653D227965732218
:100B000020747970653D22696E74222067726F755A
:100B1000703D2267656E6572616C222F3E3C726586
:100B200067206E616D653D227335222062697473A2
:100B3000697A653D22333222207265676E756D3D9C
:100B40002232312220736176652D726573746F7263
:100B5000653D227965732220747970653D22696E46
:100B600074222067726F75703D2267656E657261D1
:100B70006C222F3E3C726567206E616D653D22736D
:100B800036222062697473697A653D2233322220ED
:100B90007265676E756D3D22323222207361766513
:100BA0002D726573746F72653D22796573222074AE
:100BB0007970653D22696E74222067726F75703D91
:100BC0002267656E6572616C222F3E3C72656720FC
:100BD0006E616D653D227337222062697473697A94
:100BE000653D22333222207265676E756D3D22327B
:100BF000332220736176652D726573746F72653D63
:100C0000227965732220747970653D22696E7422A1
:100C10002067726F75703D2267656E6572616C2228
:100C20002F3E3C726567206E616D653D22733822F0
:100C30002062697473697A653D22333222207265BD
:100C4000676E756D3D2232342220736176652D7298
:100C50006573746F72653D227965732220747970B3
:100C6000653D22696E74222067726F75703D226740
:100C7000656E6572616C222F3E3C726567206E6105
:100C80006D653D227339222062697473697A653D0E
:100C900022333222207265676E756D3D2232352215
:100CA00020736176652D726573746F72653D22796C
:100CB00065732220747970653D22696E7422206705
:100CC000726F75703D2267656E6572616C222F3E92
:100CD0003C726567206E616D653D22733130222064
:100CE00062697473697A653D2233322220726567C6
:100CF0006E756D3D2232362220736176652D7265E8
:100D000073746F72653D2279657322207479706502
:100D10003D22696E74222067726F75703D2267658F
:100D20006E6572616C222F3E3C726567206E616D4C
:100D3000653D22733131222062697473697A653DA1
:100D400022333222207265676E756D3D2232372262
:100D500020736176652D726573746F72653D2279BB
:100D600065732220747970653D22696E7422206754
:100D7000726F75703D2267656E6572616C222F3EE1
:100D80003C726567206E616D653D2274332220627E
:100D9000697473697A653D22333222207265676E09
:100DA000756D3D2232382220736176652D72657330
:100DB000746F72653D227965732220747970653D88
:100DC00022696E74222067726F75703D2267656EAE
:100DD0006572616C222F3E3C726567206E616D65A5
:100DE0003D227434222062697473697A653D22332E
:100DF0003222207265676E756D3D22323922207372
:100E00006176652D726573746F72653D22796573C5
:100E10002220747970653D22696E74222067726F9A
:100E200075703D2267656E6572616C222F3E3C7263
:100E30006567206E616D653D22743522206269749C
:100E400073697A653D22333222207265676E756D53
:100E50003D2233302220736176652D726573746F85
:100E600072653D227965732220747970653D22692F
:100E70006E74222067726F75703D2267656E6572B1
:100E8000616C222F3E3C726567206E616D653D226C
:100E90007436222062697473697A653D2233322286
:100EA000207265676E756D3D223331222073617645
:100EB000652D726573746F72653D227965732220AA
:100EC000747970653D22696E74222067726F757047
:100ED0003D2267656E6572616C222F3E3C726567CC
:100EE000206E616D653D22706322206269747369B2
:100EF0007A653D22333222207265676E756D3D2220
:100F000033322220736176652D726573746F72655A
:100F10003D227965732220747970653D22696E7473
:100F2000222067726F75703D2267656E6572616C15
:100F3000222F3E3C2F666561747572653E3C666586
:100F40006174757265206E616D653D226F72672EEA
:100F5000676E752E6764622E72697363762E637393
:100F600072223E3C726567206E616D653D226D7335
:100F70007461747573222062697473697A653D22A5
:100F8000333222207265676E756D3D22383333220D
:100F900020736176652D726573746F72653D226E84
:100FA0006F2220747970653D22696E742220677209
:100FB0006F75703D22637372222F3E3C726567200D
:100FC0006E616D653D226D69736122206269747383
:100FD000697A653D22333222207265676E756D3DF8
:100FE000223833342220736176652D726573746FF5
:100FF00072653D226E6F2220747970653D22696EA4
:1010000074222067726F75703D22637372222F3EC7
:101010003C726567206E616D653D226D69652220B9
:1010200062697473697A653D223332222072656782
:101030006E756D3D223833372220736176652D72CF
:101040006573746F72653D226E6F222074797065CE
:101050003D22696E74222067726F75703D22637342
:1010600072222F3E3C726567206E616D653D226D78
:1010700074766563222062697473697A653D2233F0
:101080003222207265676E756D3D2238333822201A
:10109000736176652D726573746F72653D226E6F34
:1010A0002220747970653D22696E74222067726F08
:1010B00075703D22637372222F3E3C726567206E0D
:1010C000616D653D226D636F756E746572656E222C
:1010D0002062697473697A653D2233322220726519
:1010E000676E756D3D223833392220736176652D28
:1010F000726573746F72653D226E6F222074797011
:10110000653D22696E74222067726F75703D22639F
:101110007372222F3E3C726567206E616D653D22C1
:101120006D73637261746368222062697473697A93
:10113000653D22333222207265676E756D3D22381F
:1011400039372220736176652D726573746F72650D
:101150003D226E6F2220747970653D22696E742283
:101160002067726F75703D22637372222F3E3C724E
:101170006567206E616D653D226D6570632220623A
:10118000697473697A653D22333222207265676E15
:10119000756D3D223839382220736176652D726570
:1011A00073746F72653D226E6F2220747970653D95
:1011B00022696E74222067726F75703D22637372AC
:1011C000222F3E3C726567206E616D653D226D6326
:1011D00061757365222062697473697A653D223393
:1011E0003222207265676E756D3D223839392220B2
:1011F000736176652D726573746F72653D226E6FD3
:101200002220747970653D22696E74222067726FA6
:1012100075703D22637372222F3E3C726567206EAB
:10122000616D653D226D7476616C22206269747314
:10123000697A653D22333222207265676E756D3D95
:10124000223930302220736176652D726573746F98
:1012500072653D226E6F2220747970653D22696E41
:1012600074222067726F75703D22637372222F3E65
:101270003C726567206E616D653D226D697022204C
:1012800062697473697A653D223332222072656720
:101290006E756D3D223930312220736176652D7275
:1012A0006573746F72653D226E6F2220747970656C
:1012B0003D22696E74222067726F75703D226373E0
:1012C00072222F3E3C726567206E616D653D22740F
:1012D00073656C656374222062697473697A653D15
:1012E00022333222207265676E756D3D22323031B5
:1012F000372220736176652D726573746F72653D58
:10130000226E6F2220747970653D22696E742220EE
:1013100067726F75703D22637372222F3E3C726557
:1013200067206E616D653D227464617461312220B5
:1013300062697473697A653D22333222207265676F
:101340006E756D3D22323031382220736176652D05
:10135000726573746F72653D226E6F2220747970AE
:10136000653D22696E74222067726F75703D22633D
:101370007372222F3E3C726567206E616D653D225F
:10138000746461746132222062697473697A653DA4
:1013900022333222207265676E756D3D2232303104
:1013A000392220736176652D726573746F72653DA5
:1013B000226E6F2220747970653D22696E7422203E
:1013C00067726F75703D22637372222F3E3C7265A7
:1013D00067206E616D653D22746461746133222003
:1013E00062697473697A653D2233322220726567BF
:1013F0006E756D3D22323032302220736176652D5C
:10140000726573746F72653D226E6F2220747970FD
:10141000653D22696E74222067726F75703D22638C
:101420007372222F3E3C726567206E616D653D22AE
:1014300064637372222062697473697A653D223332
:101440003222207265676E756D3D22323033332251
:1014500020736176652D726573746F72653D226EBF
:101460006F2220747970653D22696E742220677244
:101470006F75703D22637372222F3E3C7265672048
:101480006E616D653D2264706322206269747369C8
:101490007A653D22333222207265676E756D3D227A
:1014A000323033342220736176652D726573746F28
:1014B00072653D226E6F2220747970653D22696EDF
:1014C00074222067726F75703D22637372222F3E03
:1014D0003C726567206E616D653D22647363726165
:1014E000746368222062697473697A653D223332BD
:1014F00022207265676E756D3D22323033352220B1
:10150000736176652D726573746F72653D226E6FBF
:101510002220747970653D22696E74222067726F93
:1015200075703D22637372222F3E3C726567206E98
:10153000616D653D226D6379636C6522206269741B
:1015400073697A653D22333222207265676E756D4C
:101550003D22323838312220736176652D726573F1
:10156000746F72653D226E6F2220747970653D2222
:10157000696E74222067726F75703D2263737222E8
:101580002F3E3C726567206E616D653D226D696E10
:101590007374726574222062697473697A653D227E
:1015A000333222207265676E756D3D2232383833D2
:1015B0002220736176652D726573746F72653D22AA
:1015C0006E6F2220747970653D22696E74222067E7
:1015D000726F75703D22637372222F3E3C72656795
:1015E000206E616D653D226D6379636C65682220B4
:1015F00062697473697A653D2233322220726567AD
:101600006E756D3D22333030392220736176652D41
:10161000726573746F72653D226E6F2220747970EB
:10162000653D22696E74222067726F75703D22637A
:101630007372222F3E3C726567206E616D653D229C
:101640006D696E737472657468222062697473695F
:101650007A653D22333222207265676E756D3D22B8
:10166000333031312220736176652D726573746F6A
:1016700072653D226E6F2220747970653D22696E1D
:1016800074222067726F75703D22637372222F3E41
:101690003C726567206E616D653D226379636C65A0
:1016A000222062697473697A653D22333222207286
:1016B00065676E756D3D2233313337222073617655
:1016C000652D726573746F72653D226E6F22207492
:1016D0007970653D22696E74222067726F75703D66
:1016E00022637372222F3E3C726567206E616D65C6
:1016F0003D2274696D65222062697473697A653D63
:1017000022333222207265676E756D3D223331338C
:10171000382220736176652D726573746F72653D32
:10172000226E6F2220747970653D22696E742220CA
:1017300067726F75703D22637372222F3E3C726533
:1017400067206E616D653D22696E737472657422E7
:101750002062697473697A653D2233322220726592
:10176000676E756D3D2233313339222073617665A2
:101770002D726573746F72653D226E6F22207479CD
:1017800070653D22696E74222067726F75703D220C
:10179000637372222F3E3C726567206E616D653DFA
:1017A000226379636C6568222062697473697A6563
:1017B0003D22333222207265676E756D3D223332D1
:1017C00036352220736176652D726573746F72658C
:1017D0003D226E6F2220747970653D22696E7422FD
:1017E0002067726F75703D22637372222F3E3C72C8
:1017F0006567206E616D653D2274696D65682220A4
:1018000062697473697A653D22333222207265679A
:101810006E756D3D22333236362220736176652D2A
:10182000726573746F72653D226E6F2220747970D9
:10183000653D22696E74222067726F75703D226368
:101840007372222F3E3C726567206E616D653D228A
:10185000696E737472657468222062697473697A40
:10186000653D22333222207265676E756D3D2233ED
:101870003236372220736176652D726573746F720C
:10188000653D226E6F2220747970653D22696E7409
:10189000222067726F75703D22637372222F3E3C67
:1018A000726567206E616D653D226D76656E646F51
:1018B000726964222062697473697A653D223332E9
:1018C00022207265676E756D3D22333932322220D7
:1018D000736176652D726573746F72653D226E6FEC
:1018E0002220747970653D22696E74222067726FC0
:1018F00075703D22637372222F3E3C726567206EC5
:10190000616D653D226D6172636869642220626960
:101910007473697A653D22333222207265676E7571
:101920006D3D22333932332220736176652D726525
:1019300073746F72653D226E6F2220747970653DFD
:1019400022696E74222067726F75703D2263737214
:10195000222F3E3C726567206E616D653D226D6988
:101960006D706964222062697473697A653D2233FF
:101970003222207265676E756D3D22333932342212
:1019800020736176652D726573746F72653D226E8A
:101990006F2220747970653D22696E74222067720F
:1019A0006F75703D22637372222F3E3C7265672013
:1019B0006E616D653D226D6861727469642220629A
:1019C000697473697A653D22333222207265676ECD
:1019D000756D3D22333932352220736176652D7263
:1019E0006573746F72653D226E6F22207479706525
:1019F0003D22696E74222067726F75703D22637399
:101A000072222F3E3C2F666561747572653E3C669E
:101A1000656174757265206E616D653D226F7267D8
:101A20002E676E752E6764622E72697363762E76EA
:101A300069727475616C223E3C726567206E616DDF
:101A4000653D2270726976222062697473697A65D5
:101A50003D223822207265676E756D3D2234313625
:101A6000312220736176652D726573746F72653DE6
:101A7000226E6F2220747970653D22696E74222077
:101A800067726F75703D2267656E6572616C222F9B
:101A90003E3C2F666561747572653E3C2F746172C1
:101AA0006765743E00000000348A0008608C0008FE
:101AB000608C0008608C0008608C0008608C000856
:101AC000608C0008608C0008608C0008608C000846
:101AD000608C0008608C0008608C0008608C000836
:101AE000608C0008608C0008608C0008608C000826
:101AF000608C0008608C0008608C0008608C000816
:101B0000608C0008608C0008608C0008608C000805
:101B1000608C0008608C0008608C0008608C0008F5
:101B2000608C0008608C0008608C0008608C0008E5
:101B3000608C0008608C0008608C0008608C0008D5
:101B4000608C0008608C0008608C0008608C0008C5
:101B5000608C0008608C0008608C0008608C0008B5
:101B6000608C0008608C0008608C0008608C0008A5
:101B7000608C0008608C0008608C0008608C000895
:101B8000608C0008608C00084C8A0008608C00089B
:101B9000848A0008608C0008608C0008AC8A000809
:101BA000608C0008608C0008608C0008608C000865
:101BB000608C0008608C0008608C0008608C000855
:101BC000608C0008108B0008388B0008608C0008BF
:101BD000708B0008608C0008608C0008F08B000897
:101BE0003C6D656D6F72792D6D61703E3C6D656DFC
:101BF0006F727920747970653D2272616D22207355
:101C0000746172743D223078303030303030303092
:101C100022206C656E6774683D2230783830303031
:101C2000303030222F3E3C6D656D6F7279207479B3
:101C300070653D22666C61736822207374617274F2
:101C40003D223078303830303030303022206C65F2
:101C50006E6774683D2230783230303030223E3C3E
:101C600070726F7065727479206E616D653D22626D
:101C70006C6F636B73697A65223E30783430303C28
:101C80002F70726F70657274793E3C2F6D656D6F49
:101C900072793E3C6D656D6F727920747970653D27
:101CA0002272616D222073746172743D223078302B
:101CB0003830323030303022206C656E6774683DC9
:101CC0002230786637666530303030222F3E3C2F28
:101CD0006D656D6F72792D6D61703E0025303278C3
:101CE00000000000E4A5000838A7000838A7000895
:101CF00038A7000838A7000838A7000838A7000848
:101D000038A7000838A7000838A7000838A7000837
:101D100038A7000838A7000838A7000838A7000827
:101D200038A7000838A7000838A7000838A7000817
:101D300038A7000838A7000838A7000838A7000807
:101D400038A7000838A7000838A7000838A70008F7
:101D500038A7000838A7000838A7000838A70008E7
:101D600038A7000838A7000838A7000838A70008D7
:101D700038A7000838A7000838A7000838A70008C7
:101D800038A7000838A7000838A7000838A70008B7
:101D900038A7000838A7000838A7000838A70008A7
:101DA00038A7000838A7000838A7000838A7000897
:101DB00038A7000838A7000838A7000838A7000887
:101DC00038A7000838A7000838A7000838A7000877
:101DD00038A7000838A7000838A7000838A7000867
:101DE00038A7000838A7000838A7000838A7000857
:101DF00038A7000838A7000838A7000838A7000847
:101E000038A7000838A7000838A7000838A7000836
:101E100038A7000838A7000838A7000838A7000826
:101E200038A7000838A7000838A7000838A7000816
:101E300038A7000838A7000838A7000838A7000806
:101E400038A7000838A7000838A7000838A70008F6
:101E500038A7000838A7000838A7000838A70008E6
:101E600038A7000838A7000838A7000838A70008D6
:101E700038A7000838A7000838A7000838A70008C6
:101E800038A7000838A7000838A7000838A70008B6
:101E900038A7000810A4000838A7000838A70008D1
:101EA00038A7000838A7000838A7000838A7000896
:101EB00034A5000838A7000838A7000838A700088C
:101EC00038A7000838A7000838A7000838A7000876
:101ED00038A7000880A5000838A7000838A7000820
:101EE00038A7000838A7000838A7000838A7000856
:101EF00038A7000824A4000838A7000838A700085D
:101F000048A4000838A7000838A7000838A7000828
:101F100038A70008D4A5000838A7000804A60008C0
:101F200038A7000820A6000838A700083CA600082B
:101F300038A7000858A6000838A7000874A60008AB
:101F400038A7000890A6000838A70008ACA600082B
:101F500038A70008C8A6000838A70008E4A60008AB
:101F600038A7000800A7000838A700081CA7000829
:101F700038A70008D8A400082578000051537461E0
:101F800072744E6F41636B4D6F6465005A25782CF7
:101F900025782C257800000071537570706F72746D
:101FA00065643A0071586665723A66656174757267
:101FB00065733A726561643A7461726765742E780C
:101FC0006D6C3A0071586665723A6D656D6F727925
:101FD0002D6D61703A726561643A3A007152636DB9
:101FE000642C0000726573657400000068616C7495
:101FF00000000000756E737570706F7274656420F8
:102000006D6F6E69746F7220636F6D6D616E642E9B
:102010000A0000005330320076466C6173684572E6
:102020006173653A0000000076466C617368577210
:102030006974653A0000000076466C617368446F0D
:102040006E6500007A25782C25782C257800000014
:1020500054303200543035004525303278000000CD
:102060004F4B00005061636B657453697A653D3472
:1020700030353B5153746172744E6F41636B4D6FD9
:1020800064652B3B71586665723A6665617475725A
:1020900065733A726561642B3B71586665723A6D7F
:1020A000656D6F72792D6D61703A726561642B0098
:1020B000232D302B20000000686C4C0065666745BE
:1020C00046470000303132333435363738394142F3
:1020D0004344454600000000303132333435363752
:1020E000383961626364656600000000412D466115
:1020F0002D66383930313233343536375D000000E3
:102100002B2D000030300000785800000000000047
:1021100000000000000000000000000000000000BF
:1021200000000000000000000000000000000000AF
:10213000000000000000000000000000000000009F
:10214000000000000000000000000000000000008F
:10215000000000000000000000000000000000007F
:10216000000000000000000000000000430000002C
:10217000504F5349580000002E000000002020203E
:102180002020202020202828282828202020202027
:1021900020202020202020202020202020881010F7
:1021A0001010101010101010101010101004040453
:1021B0000404040404040410101010101010414111
:1021C00041414141010101010101010101010101FF
:1021D0000101010101010101101010101010424213
:1021E00042424242020202020202020202020202CF
:1021F000020202020202020210101010200000006F
:1022000000000000000000000000000000000000CE
:1022100000000000000000000000000000000000BE
:1022200000000000000000000000000000000000AE
:10223000000000000000000000000000000000009E
:10224000000000000000000000000000000000008E
:10225000000000000000000000000000000000007E
:10226000000000000000000000000000000000006E
:10227000000000000000000000000000000000005E
:10228000130101FF23261100EF00403913057005EB
:10229000EF00C007EF0000268320C10013010101F9
:1022A00067800000678000006F000000B717000023
:1022B0009387F7FF6304F5006F000000130101FF2F
:1022C00023261100EFF05FFE6F000000B70700202B
:1022D00003A787663305A700938781786360F502BB
:1022E000B78700209387078063EEA700B707002019
:1022F00023A4A76613050700678000001307F0FFFB
:102300006FF05FFF1307F0FF6FF0DFFEB70700D23B
:1023100023800700A385070013154500B71700D2D7
:102320003385A70063F8A70023A007009387070160
:102330006FF05FFF6780000013152500B71700D20C
:10234000938717003305F500930710002300F5006D
:102350006780000013152500B71700D29387370058
:102360003305F5002300B500678000001315250034
:10237000B71700D2938737003305F50003450500F2
:1023800067800000B70700D22380A70067800000A5
:10239000B70700D203C5070067800000130101FFE3
:1023A0002326110023248100131515001374F50F43
:1023B000EFF01FFE1375150E1374E40133658500ED
:1023C000EFF05FFC8320C1000324810013010101B1
:1023D00067800000130101FF23261100EFF05FFB6F
:1023E000135515001375F5008320C1001301010179
:1023F00067800000130101FF2326110023248100C0
:1024000023229100232021011309050013840500D4
:10241000EFF05FFC930405009307400063F4A7000E
:102420009304400093078000B38797403314F4006F
:102430001374F40F13050900EFF05FF3B315950063
:1024400093F5F50FB3D5954093F5F50FB365B4004B
:1024500013050900EFF01FF08320C1000324810061
:10246000832441000329010013010101678000005A
:10247000130101FF23261100232481002322910050
:10248000232021011309050013840500EFF09FF4B8
:102490009307300063F2A702130400001305040041
:1024A0008320C1000324810083244100032901000B
:1024B0001301010167800000930405001314440018
:1024C0001374F40F13050900EFF05FEA9305800021
:1024D000B3849540B355954093F5F50FB3959500AA
:1024E00093F5F50FB365B40013050900EFF09FE60F
:1024F0006FF0DFFAF327503093F707FC93E73700CC
:102500007390573067800000371702408327070019
:10251000B7060100B3E7D7002320F70093070000B8
:102520009387170037170240032707009316E70029
:1025300063C80600370701001307F7FFE392E7FEC1
:10254000B717024083A707001397E700634407000B
:102550006F000000B717024003A7470023A2E7005F
:1025600003A7470023A2E70003A74700136707401C
:1025700023A2E70003A74700B706C4DF9386F6FF50
:102580003377D70023A2E70003A74700B7061D2033
:102590003367D70023A2E70003A7C702B7F6FEFF01
:1025A0003377D70023A6E70203A7C70213671700F4
:1025B00023A6E70203A70700B70600013367D70089
:1025C00023A0E700B717024083A70700139767000F
:1025D000E35A07FEB717024003A747001377C7FF68
:1025E00023A2E70003A747001367270023A2E70001
:1025F000B717024083A7470093F78700E38A07FED7
:1026000067800000130101FF23261100EFF0DFEFC8
:102610008320C1001301010167800000130101FF45
:1026200023261100B717024003A7070013671700FE
:1026300023A0E70003A74700B706FFE09386C60084
:102640003377D70023A2E70003A70700B706F7FEFA
:102650009386F6FF3377D70023A0E70003A7070090
:10266000B706FCFF9386F6FF3377D70023A0E70079
:1026700003A74700B70601DF9386F6FF3377D7003D
:1026800023A2E70023A6070203A70700B706F7EA7D
:102690009386F6FF3377D70023A0E7003707FF00C4
:1026A00023A4E700EFF01FF68320C100130101010E
:1026B0006780000093F8F50093F705016384070035
:1026C000B3E8C800930700006F008001232AE500EB
:1026D0002320C500938717009397070193D707011D
:1026E000130770006366F704130710003317F70031
:1026F0003377D700E30007FE032305001398270074
:102700001306F000331606011346F6FF3376660013
:10271000339808013366C80013088002E38805FB7C
:1027200013088004E39605FB2328E5006FF05FFAA9
:10273000930780006F008001232AC5002322E50053
:10274000938717009397070193D707011307F000AA
:10275000636CF704130610003316F6003376D600C8
:10276000E30006FE0323450037070040130787FFF9
:102770003387E700131727001308F0003318E80029
:102780001348F8FF337868003397E8003367070190
:1027900013088002E38205FB13088004E39005FB25
:1027A0002328C5006FF09FF9678000002328B5003B
:1027B00067800000232AB50067800000832785001A
:1027C000B3F5B700638605001305100067800000AD
:1027D000130500006780000093576500371702401B
:1027E000B387E70003A7070093061000B396A6007F
:1027F0003367D70023A0E700678000009357650088
:1028000037170240B387E70003A7070093061000BD
:10281000B396A6003367D70023A0E70067800000C7
:1028200013576500B71702403307F70083260700E8
:1028300093071000B397A70093C7F7FFB3F7F6000D
:102840002320F70067800000B716024083A74600E8
:10285000370740FF1307F7FFB3F7E70033E5A7009B
:1028600023A2A60067800000130101FD23261102A8
:102870002324810223229102232021031304050033
:10288000B70700089387072403A6070083A647001D
:1028900003A7870083A7C7002328C100232AD100EC
:1028A000232CE100232EF10003A781812324E100E2
:1028B0009387818183A747002326F1002320E1002D
:1028C0002322F100B717024083A7470093D72700C0
:1028D00093F7370013072000638EE708B7167A00D6
:1028E00093860620371602408327460093D7470079
:1028F00093F7F70013070102B307F70003C707FFB9
:1029000033D7E6008327460093D7870093F77700F5
:1029100093050102B387F50083C787FEB355F7001F
:102920008327460093D7B70093F777001306010279
:10293000B307F60083C707FE3355F700930710006F
:102940006308F412630A041293072000630AF41266
:10295000930730006304F400130500008320C102D4
:10296000032481028324410203290102130101038C
:1029700067800000B717024083A747001397F7004E
:10298000635E070CB717024083A7C7021397F700CF
:102990006350070CB717024083A5C70293D54500C3
:1029A00093F5F5009385150083A4C70293D48400A2
:1029B00093F4F40093842400930710016386F408D1
:1029C00037157A0013050520EF70507E93850400BB
:1029D000EF70107BB717024083A5C70293F5F5008F
:1029E00093851500EF70907C13090500B71702401E
:1029F00003A54700135525011375F50083A747006C
:102A00001397270063540700136505019307E0003F
:102A100063ECA704930425009305090013850400C3
:102A2000EF701076930605009307F000E39CF4EA3C
:102A300093171900B38727019396170013591900AC
:102A4000B38626016FF01FEA930440016FF05FF731
:102A500037157A00130505206FF0DFF737193D00B1
:102A6000130909906FF09FF8930415006FF0DFFAD7
:102A7000130507006FF09FEE138506006FF01FEE41
:102A8000138505006FF09FED130101FF2326110050
:102A9000B7170040938707C06300F50CB7170040D5
:102AA000938707C063E8A702B707004093870740F2
:102AB0006300F508B7170040938707806304F508A3
:102AC000B7070040630CF5048320C1001301010126
:102AD00067800000B7170040938707406308F50838
:102AE000B7370140938707C06300F502B71700406E
:102AF000E31CF5FC13054040EFF05FD013054040A8
:102B0000EFF01FD26FF05FFC1305B030EFF01FCF76
:102B10001305B030EFF0DFD06FF01FFB130500405E
:102B2000EFF0DFCD13050040EFF09FCF6FF0DFF93E
:102B300013051040EFF09FCC13051040EFF05FCE6F
:102B40006FF09FF813052040EFF05FCB1305204096
:102B5000EFF01FCD6FF05FF713053040EFF01FCAA5
:102B600013053040EFF0DFCB6FF01FF61305504038
:102B7000EFF0DFC813055040EFF09FCA6FF0DFF4AD
:102B800083D705002324F502B7370140938707C098
:102B90006308F504B70700406304F5049387074012
:102BA0006300F504B717004093870780630AF502B6
:102BB000B7170040938707C06304F5028327050019
:102BC00093F7F7FE2320F5008327050003D7450080
:102BD00013770701B3E7E7002320F5006F008003B8
:102BE0008327050093F7F7F82320F50083270500D6
:102BF00003D7250013770706B3E7E7002320F50086
:102C00008327050003D7450013770701B3E7E700E3
:102C10002320F50083A785002326F502B71700407F
:102C20006306F502938707406302F50283270500D8
:102C300093F7F7CF2320F5008327050003D7C500BE
:102C400013770730B3E7E7002320F500B7370140DB
:102C5000938707C0630AF5008327450193E71700B0
:102C6000232AF5006780000083C7E5002328F502CA
:102C70006FF09FFE8327050093E717002320F500E0
:102C8000678000008327050093F7E7FF2320F50006
:102C9000678000008327050093F7D7FF2320F50006
:102CA0006780000093074000638CF500639805007F
:102CB0008327050093F7B7FF2320F5006780000006
:102CC0008327050093E747002320F5006780000075
:102CD0008327C500B3E5B7002326B5006780000051
:102CE00083270501B3F5B7006386050013051000BF
:102CF00067800000130500006780000093C5F5FFA2
:102D00002328B50067800000F36704306780000067
:102D1000130101FF232611001375F50FEFF00FE8E3
:102D20008320C1001301010167800000130101FF2E
:102D30002326110023248100232291002320210136
:102D4000130405001389050093040600EFF0CFDE9D
:102D50009305090013050400EFF0CFE99385040003
:102D600013050400EFF0CFF08320C100032481009D
:102D70008324410003290100130101016780000041
:102D8000B707014083A607401347F5FFB3F6E600F7
:102D900023A0D74083A64740B376D70023A2D740CD
:102DA00083A68740B376D70023A4D74083A6C74025
:102DB000B376D70023A6D74063820502930710009D
:102DC0006388F50293071000630EF604630C060295
:102DD000930720006308F60667800000B7060140ED
:102DE00083A70640B3E7A70023A0F6406FF09FFD3E
:102DF000B706014083A74640B3E7A70023A2F640E9
:102E00006FF05FFCB707014083A6874033E5A6005B
:102E100023A4A74083A6C7403377D70023A6E74063
:102E200067800000B707014083A687403377D7004B
:102E300023A4E74003A7C7403365A70023A6A74004
:102E400067800000B707014003A787403367A700EA
:102E500023A4E74003A7C7403365A70023A6A740E4
:102E600067800000370701408327074033E5A7004C
:102E70002320A74067800000B707014023AAA7408E
:102E800067800000B777004003A707001377C7FFEC
:102E900023A0E70003A707003365A70023A0A7002E
:102EA000F3E710816398050073005010F3F7108169
:102EB00067800000F3770430F3E70081730050105F
:102EC000F3F70081F36704306FF05FFE130101FF39
:102ED00023261100032705008327070193E7170026
:102EE0002328F7008327050083A7070193F717001E
:102EF000E39A07FE13053000EF20D0188320C100AD
:102F00001301010167800000130101FE232E11004F
:102F1000232C8100232A910023282101232631011B
:102F200023244101232251012320610123020500B2
:102F300093072000A300F5002300C500630A0600E4
:102F4000930710006304F60C130510006F00401384
:102F50009307C0002301F50093076000A301F5006B
:102F600093072000A302F5003709044013840500ED
:102F700093040500930710002303F500A303F50055
:102F8000B7170000138B0780330B6901930A0940C0
:102F9000130A0944938707E0B309F9001306C00B2D
:102FA0009305000013050400EF70903823202401DE
:102FB0002322640123245401232C4407232C340BA3
:102FC0001307000083C734006372F7069317570096
:102FD000B3872701B716000093850690B385B70025
:102FE000131627003306C4002326B600938606B0C6
:102FF000B387D7009306870093962600B306D400C4
:1030000023A2F600130717006FF0DFFB9307800081
:103010002301F50093074000A301F500930720006A
:10302000A302F500370900506FF05FF4930700002A
:1030300003C7240063F4E70493965700B386260180
:10304000938606501387C700131727003307E40041
:103050002326D7009396C700B386260137170000B2
:10306000B386E6001387C701131727003307E40070
:103070002326D700938717006FF09FFB13050000EE
:103080008320C1010324810183244101032901011B
:103090008329C100032A8100832A4100032B0100F8
:1030A0001301010267800000130101FE232E1100AD
:1030B000232C81002324A1002326B1001304060041
:1030C0008327060003A7870303A787001377E7FF7B
:1030D00023A4E7000347D10093071000630CF70413
:1030E000032706008327C70093E707042326F7007A
:1030F00013050600EFF09FDD8347E10063900708AA
:1031000037072D008327040023ACE7021305400195
:10311000EF2000790347C100930710006304F7060E
:10312000130500008320C101032481011301010262
:1031300067800000832706003707100023ACE702F2
:103140008326060083A7C6003707E0FF1307F7FBB7
:10315000B3F7E70023A6F6008326060083A7C60080
:103160003707F0FF1307F7FFB3F7E70023A6F600D2
:1031700013050600EFF09FD56FF0DFF937073D002C
:103180006FF05FF8032704008327870093E70702A7
:103190002324F700032704008327870093F717FEF3
:1031A0002324F700032704008327870093E7A70061
:1031B0002324F7006FF0DFF69386360093D62600BF
:1031C0001306C601131626003306C5000325C600E4
:1031D0001386F6FF638E060283C7050003C715003A
:1031E00013178700B3E7E70003C72500131707018C
:1031F000B3E7E70003C7350013178701B3E7E7001C
:103200002320F50093854500930606006FF05FFCD0
:1032100013050000678000001306360013562600D1
:103220000325C5071307F6FF630806028327050079
:103230002380F50093D68700A380D50093D607019D
:103240002381D50093D78701A381F500938545009D
:10325000130607006FF01FFD13850500678000004F
:10326000130101FF232611009395650083270500B4
:1032700093E5050223A8B7008327050083A707016C
:1032800093F70702E39A07FE13053000EF20805FF3
:10329000130500008320C1001301010167800000B5
:1032A000130101FF232611008327050013070001E6
:1032B00023A8E7008327050083A7070193F70701E9
:1032C000E39A07FE13053000EF20C05B13050000F2
:1032D0008320C1001301010167800000832785005E
:1032E0001307F0FF23A2E70003278500B70700C0FC
:1032F0009387F7FF232AF70003278500B71700807D
:1033000093870780232CF70083474500639A0700C3
:10331000032785008327870193E70701232CF70004
:103320008326850083A7860137370C001307A70083
:10333000B3E7E70023ACF600032785008327870067
:1033400093E717002324F7001305000067800000AF
:10335000130101FF23261100232481002322910061
:10336000130405008326850083A7C600370700A045
:103370001307F7FFB3F7E70023A6F600032785003E
:103380008327C700B7060040B3E7D7002326F7001E
:103390008327050C23A007008326C50083A706000A
:1033A00037E7FFFF1307F77FB3F7E70023A0F60027
:1033B0008327C50003A7070023A0E7000327C50054
:1033C0008327070093F7C7FF2320F7000347050073
:1033D000930710006304F70493048400930500012D
:1033E00013850400EFF0DFE713850400EFF05FEBD7
:1033F0008327C40023A807008327C40023AA07004B
:103400008327C4001307F0FF23ACE7008327C40021
:1034100023AE0700930700006F00400D0327C5008F
:103420008327070093E737002320F70083278500D1
:103430001307000823A2E70203278500B70740000F
:10344000938707082324F702930500081307100049
:1034500093073000E3E2E7F89306F7FFB7D70008D9
:10346000938747E493961600B386D70083D6060069
:10347000B385D50093161700B387D70083D707000D
:103480009397070183268400B3E7B7001306F70379
:1034900013162600B386C60023A2F60013071700F2
:1034A0006FF01FFB8326070037060048B3E6C6000F
:1034B0002320D7006F0080058326070037060048C9
:1034C000B3E6C6002320D700138787001317270011
:1034D0003307E4008326C70023A806000327C7009C
:1034E0009306F00F2324D700938717000347340077
:1034F00063FCE704139727003307E4000327470121
:1035000083260700E3C006FA23200700139727004D
:103510003307E4008326470123A806000327470159
:103520009306F00F2324D700138787001317270073
:103530003307E4000327C70083260700E3CE06F61F
:10354000232007006FF05FF813050400EFF01FD988
:10355000130500008320C10003248100832441005F
:1035600013010101678000000327C500832747007E
:1035700093E727002322F700678000000327C50098
:103580008327470093F7D7FF2322F70067800000C7
:103590000327C5008327070093F7F7802320F70050
:1035A0000327C5008327070093954500B3E7B700BD
:1035B0002320F70067800000130101FF232601008C
:1035C00083A7050093F7F70013880700038705001A
:1035D000634A070A13878700131727003307E5009C
:1035E0000327C7001386070193061000B396C60091
:1035F0002326D1008326070013960601634406069E
:1036000083260700370634FC13060680B3F6C6008F
:103610002320D700631608088326C50083A68600EA
:1036200013F8660003260700B7D60008938606E461
:10363000B386060183C60600B366D6002320D700F2
:103640008326070003C6150013162601939767010A
:10365000B367F600B3E6F600B7870010B3E6F600EE
:103660002320D7008326C1000327C5008327C70175
:10367000B3E7D700232EF700130500001301010163
:1036800067800000139727003307E50003274701F1
:1036900093061000B396F6002326D1006FF09FF535
:1036A0008326070003D64500B3E6C6002320D700D3
:1036B0006FF01FF983A7050093F7F7000387050054
:1036C0006348070493860701130710003317D700D8
:1036D0009387870093972700B307F50003A6C700D9
:1036E00083270600B786FFFF9386F6FFB3F7D70060
:1036F0002320F6008326C50083A7C6011347F7FFE2
:1037000033F7E70023AEE6001305000067800000F2
:10371000130710003317F70093972700B307F5003E
:1037200003A6470183270600B786FFFF9386F6FFAF
:10373000B3F7D7002320F6006FF0DFFB130101FE83
:10374000232E1100232C8100232A910023282101FC
:10375000130905001384050083A4050093F4F40005
:1037600093972400B307F50083A7470103A7070039
:103770002326E10083A707012324F100832781008A
:10378000370700E0B3F7E7002324F10003A5C500E5
:103790006316050A8327810037070800B3E7E700AF
:1037A0002324F10093972400B307F90083A747016E
:1037B0000327810023A8E70003474900930710006F
:1037C000630AF70E03471400930710006300F71015
:1037D0008327C10037070084B3E7E7002326F10001
:1037E00093972400B307F90083A747010327C1007B
:1037F00023A0E70003471400930710006304F710A9
:103800008327C400638E07008326C90083A746036D
:1038100013071000B3149700B3E4970023AA96028D
:10382000130500008320C101032481018324410189
:10383000032901011301010267800000639A040457
:1038400083D7450063F4A700138507002326A4004F
:103850008327810037070800B3E7E7002324F1003E
:103860008327C40003278100B3E7E7002324F10086
:103870000347140093071000E316F7F28327810033
:1038800037070060B3E7E7002324F1006FF09FF1F2
:1038900083D545003305B5001305F5FFEF70001122
:1038A00013153501832781003365F5002324A1001A
:1038B0006FF01FFB93972400B307F90083A747011C
:1038C0000327840123AAE7006FF0DFEF8327C900F5
:1038D00083A7870093F70710638C07008327C10035
:1038E00037070020B3E7E7002326F1006FF05FEE13
:1038F0008327C10037070010B3E7E7002326F10054
:103900006FF01FED8356C4001386040083258400E6
:1039100013058900EFF05F8A6FF09FF0130101FD3E
:103920002326110223248102232291022320210332
:10393000232E3101232C4101232A51012328610127
:1039400023267101930405009389050003A4050053
:103950001374F4009307840093972700B307F500CE
:1039600083AAC70003AA0A0003A50A01370900E0D9
:10397000337B250103A5C50063040500631E04060F
:1039800003D5490033656501B70708003365F500C5
:1039900023A8AA0003C74400930710006306F70892
:1039A00003C7190093071000630EF708B7070084D8
:1039B000336AFA001304840013142400338484004F
:1039C0008327C40023A04701130500008320C10200
:1039D0000324810283244102032901028329C101B6
:1039E000032A8101832A4101032B0101832BC1009A
:1039F000130101036780000083DB45003305750177
:103A000093850B001305F5FFEF60507A93050500D1
:103A1000131935013369690113850B00EF60507686
:103A2000336525016FF0DFF6930784009397270035
:103A3000B387F40083A7C70003A7890123AAE7007F
:103A40006FF01FF683C7390063880700B7070020AF
:103A5000336AFA006FF09FF5B7070010336AFA0077
:103A60006FF0DFF483A7050093F7F70003870500E5
:103A7000634607029387870093972700B307F500F3
:103A800003A7C70083270700B7062000B3E7D700C6
:103A90002320F7001305000067800000939727009C
:103AA000B307F50083A747011387070083A6070024
:103AB000E3DA06FC83A6070037060040B3E6C6003B
:103AC00023A0D7006FF01FFC83A7050093F7F70032
:103AD00003870500634207049387870093972700B5
:103AE000B307F50083A6C70083A706003707E0FFEA
:103AF0001307F7FFB3F7E70023A0F60083C715000D
:103B00009387E7FF93F7F70F13071000637EF70023
:103B1000130500006780000093972700B307F500A6
:103B200083A647016FF05FFC83A7060037070010EC
:103B3000B3E7E70023A0F6006FF09FFD8327C500E1
:103B400003A5870183A7C7013375F5001355050148
:103B50001375F50367800000938585009395250014
:103B6000B305B50083A7C50003A787008327C50059
:103B700003A547013375A700678000008327C500B0
:103B800003A5870183A7C7013375F5001375F503F6
:103B9000678000000327C5008326070183274703AA
:103BA000B3D7B7009397770093F7F70FB3E7D70032
:103BB000939525003305B5000327450103258700AC
:103BC0003375F500678000000327C502B70708605A
:103BD000938787012328F7000347450093071000C8
:103BE0006304F70067800000130745428327C5027E
:103BF00023AAE7000327C50283270700B7860080B2
:103C0000B3E7D7002320F7006FF0DFFD834775008F
:103C1000638207028327C50083A7870093F71700F5
:103C2000638A07000327050C8327070093F7C7FF64
:103C30002320F700678000000327850083274701C2
:103C400093F717006398071A130101FF2326110049
:103C50002324810023229100032447018327870125
:103C60003374F40063040410930405009317C40034
:103C700063C807109317D40063C80710B717000074
:103C800093870780B377F40063960710634A0410A4
:103C9000937724006388070083A78400130720001C
:103CA00023AAE70093778400638E070483A7044365
:103CB00083A787016386070013850400E780070058
:103CC000B707002083C7876893F7F70F638607025B
:103CD000B70700209387876803C7070013071700FB
:103CE0001377F70F2380E70083C7070093F7F70FD9
:103CF000130720006364F70C83A784001307800078
:103D000023AAE700937704016394070C9317340107
:103D100063C6070C9317240163C8070C9317B400FC
:103D200063D2070283A7044383A7C7016386070002
:103D300013850400E780070083A78400370710007D
:103D400023AAE7009317A40063D2070283A70443C2
:103D500083A707026386070013850400E780070036
:103D600083A784003707200023AAE7008320C1002F
:103D700003248100832441001301010167800000B6
:103D8000EF0080076FF01FEF13850400EF00401D68
:103D90006FF0DFEE13850400EF0080616FF01FEF1E
:103DA00083C7740C93F7F70F2383F40C83A7840065
:103DB0003707008023AAE7006FF09FED138504000A
:103DC000EF10C059B7070020238407686FF0DFF2B7
:103DD00013850400EF0080286FF05FF31385040063
:103DE000EF00003D6FF01FF313850400EF0040511A
:103DF0006FF0DFF267800000130101FD232611023E
:103E0000232481022322910223202103232E310126
:103E100013090500EFF09FD213040500930400007E
:103E20006F0000079387840093972700B307F9007A
:103E300083A7C70083A707012326F1001397340047
:103E40003307974093172700B307F90003D70727D5
:103E50008326C100370608001306F6FFB3F6C60036
:103E60003307D74023AEE7266F004007639404086A
:103E70000347C94293076000631EF7061305090054
:103E8000EFF09FD46F0000071354140093841400C4
:103E90006308040A93771400E38807FE93F9F40F8C
:103EA0009385090013050900EFF01FCB2324A1001F
:103EB0008327810093F71700638E0702938784009E
:103EC00093972700B307F90003A7C70093071000D3
:103ED0002324F70003474900E306F7F4938509001C
:103EE00013050900EF1080520347490093071000A3
:103EF000E30EF7F68327810093F78700E38607F840
:103F0000E39404F8B707002083C7876893F7F70F97
:103F1000E38C07F613050900EF104044B7070020B3
:103F2000238407689387840093972700B307F900D9
:103F300083A7C7001307800023A4E7006FF0DFF416
:103F4000130510008320C10203248102832441024F
:103F5000032901028329C1011301010367800000C5
:103F6000130101FD23261102232481022322910241
:103F700023202103232E3101232C410113090500A5
:103F8000EFF0DFBF13040500930400006F0000058D
:103F900093972400B307F90083A74701130A100081
:103FA00023A447019385090013050900EF10C057AA
:103FB00083474900639A4705639804040347C9424D
:103FC000930750006312F70413050900EFF0DFBFF9
:103FD0006F0080031354140093841400630E0404D0
:103FE00093771400E38807FE93F9F40F9385090093
:103FF00013050900EFF01FBA2326A1008327C10093
:1040000093F71700E39607F88327C10093F7070893
:10401000E38207FC9385040013050900EF00804547
:1040200093972400B307F90083A7470113070008FB
:1040300023A4E7006FF01FFA130510008320C102CC
:104040000324810283244102032901028329C1013F
:10405000032A81011301010367800000130101FDA0
:1040600023261102232481022322910223202103EB
:10407000232E3101232C4101930405002326010046
:10408000032785008327870193F7F7FE232CF7008A
:104090008327850083A707022326F1000329C10097
:1040A0001379F9000326C100135646001374F67FF6
:1040B0008327C10093D7F70013F737008327C10088
:1040C00093D7170193F7F700930620006380D70476
:1040D00093066000638CD70603A7840083278701BB
:1040E00093E70701232CF700130510008320C1027A
:1040F0000324810283244102032901028329C1018F
:10410000032A81011301010367800000E30604FC18
:10411000131A3900B3072A4193992700B3093501CF
:104120001306040083A5492713058500EFF0CF8E01
:1041300083A74927B387870023AAF92603A6C9279F
:104140003306860023AEC9266FF01FF99316390097
:10415000B386264193972600B307F50083C7C72689
:1041600093F7F700E39A07F693078000E316F4F657
:10417000E31407F613060400930545421305850072
:10418000EFF08F8993173900B386274113972600E4
:104190003387E4000326C72733068600232EC7266D
:1041A000B7070020130710002384E7686FF0DFF2E1
:1041B000130101FF232611002324810023229100F3
:1041C00023202101130405000327C500832747008E
:1041D00093F7E7FF2322F7009305000013058500FE
:1041E000EFF00F881307000083473400637AF7026B
:1041F00093172700B307F40083A747019306F00F36
:1042000023A4D7009307870093972700B307F400F0
:1042100083A7C70023A4D700130717006FF0DFFCA4
:104220008327C4001307F0FF23ACE7000327C40073
:10423000B707010093871700232EF7008327C400D8
:104240001307900023AAE7008327C40093041000FB
:1042500023A897000327C4008327070093F7F7805C
:104260002320F700A302040C13050400EFF0DF95F0
:10427000832784003717000023AAE700232604269B
:1042800023280426232A0426232C0426232E04264E
:104290002320042823220428130900042318242798
:1042A0009305C42613050400EFF00FB12324040C7A
:1042B0002326040C2328040C232A040C232C040C8E
:1042C000232E040C2320040E930700F82304F40C7F
:1042D0002316240D9305840C13050400EFF0CFADD5
:1042E0002303940C130510008320C10003248100D4
:1042F00083244100032901001301010167800000AC
:104300008326C50083A7860093D7170013F73700CD
:1043100083A7460093F7F7EF23A2F6008326C50094
:1043200083A7460093E7071023A2F6000326850023
:104330008327C600B7C6FFFF9386F63FB3F7D700C3
:104340002326F600B7D700089387C7E4B387E700B2
:1043500003C7070093073000630CF70293072000A0
:10436000A300F5008326850083A7C6003717000049
:1043700013070740B3E7E70023A6F600832785006D
:104380003727000023AAE70013051000678000000C
:10439000A300F5008326850083A7C6003727000009
:1043A00013070740B3E7E70023A6F6006FF01FFDF1
:1043B000130101FE232E1100232C8100130405009C
:1043C00083477500A307F1008327C50083A78700F3
:1043D00093F717002307F1008347650C93F7F70F56
:1043E000130730006384E70693070000A306F1007B
:1043F0008347640C93F7F70FA303F40C9307400073
:104400002303F40C8347F10093F7F70F638E070043
:104410008347E10093F7F70F638807008347D100D4
:1044200093F7F70F6398070203278400B71700007C
:1044300093870780232AF700130510008320C1010A
:10444000032481011301010267800000930710001B
:104450006FF0DFF90327040C8327070093E7370089
:104460002320F7009305000013051000EFE09FA143
:104470006FF09FFB130101FE232E1100232C8100FE
:10448000232A9100232821012326310123244101DD
:104490009309050013890500139735003307B740CA
:1044A00093172700B307F50003A7470D83A6870DD1
:1044B0003307D74003DAC70C6364EA00130A070026
:1044C000130A3A00135A2A006F004005138A340079
:1044D000135A2A0093173900B387274113942700F2
:1044E000338489009396040193D606011376F90F5D
:1044F0008325040D13858900EFE01FCC8327040D6D
:10450000B38797002328F40C8327840DB384F40029
:10451000232C940C8327440D6380F4069317290001
:10452000B387F90083A7470183A787019397070102
:1045300093D707016372FA0613173900330727412F
:1045400093172700B387F90003A7870D83A7470DAB
:104550006374F704B387E74093163900B3862641A6
:10456000139726003387E9008354C70CE3E0F4F681
:10457000938407006FF09FF583A6C90003A7460345
:1045800093071000B397270193C7F7FFB377F7009E
:1045900023AAF6026FF09FF8130510008320C101D3
:1045A0000324810183244101032901018329C100DE
:1045B000032A81001301010267800000130101FF3B
:1045C0002326110003C7250003C8450083C75500F3
:1045D0009397870033E807019317870193D78741A3
:1045E00063C2070813163700B306E6409397260008
:1045F0009386070093870726B307F5009387C700C4
:10460000B306D50003C6C6261376F6072386C6264C
:104610001377F70083C6070093F606FF33E7E6003B
:104620002380E7001377F80F2392E70003C73500D4
:10463000137737009316270037070008130707255D
:104640003307D70003270700A380E70093850700FF
:10465000EFE09FF6130500008320C1001301010164
:10466000678000009378F70713963800B307164168
:10467000939627009386060CB306D5009387860091
:104680003306164193162600B306D50003C6860CE2
:10469000136606F82384C60C6FF09FF7130101FF21
:1046A000232611009397850193D7874163C807029A
:1046B00093973500B385B7409397250093850726D8
:1046C000B305B5009385C500EFE0DFFE13050000DC
:1046D0008320C100130101016780000093F5F507F5
:1046E00093973500B387B740939527009385050CC2
:1046F000B305B500938585006FF01FFD130101FF21
:104700002326110013F8F50713173800B3050741E6
:104710009397250093870726B307F5009385C70075
:104720003307074193172700B307F50023AAC726CD
:1047300023ACD72623AE0726034745009307100076
:10474000630CF700EFF08F9D130500008320C1007C
:104750001301010167800000931738003388074177
:1047600093172800B307F50023A2C7286FF09FFD19
:10477000130101FF2326110013F8F5071317380062
:10478000B3050741939725009387070CB307F500FE
:10479000938587003307074193172700B307F50078
:1047A00023A8C70C23AAD70C23AC070C034745004A
:1047B00093071000630CF700EFE05FF813050000AB
:1047C0008320C100130101016780000093173800A6
:1047D0003388074193172800B307F50023A0C70EBD
:1047E0006FF09FFD130101FF2326110093978501B0
:1047F00093D7874163CC070293973500B385B740C1
:104800009397250093850726B305B5009385C500CA
:10481000930710002381F500EFF0CFA413050000EB
:104820008320C100130101016780000093F5F507A3
:1048300093973500B387B740939527009385050C70
:10484000B305B500938585006FF09FFC130101FF50
:10485000232611009397850193D7874163CA0702E6
:1048600093973500B385B740939725009385072626
:10487000B305B5009385C50023810500EFF0CFA4F3
:10488000130500008320C1001301010167800000AF
:1048900093F5F50793973500B387B74093952700B5
:1048A0009385050CB305B500938585006FF0DFFC9B
:1048B000130101FF23261100EFE09FCD8320C100EB
:1048C000130101016780000093973500B385B7405D
:1048D000939725003305F5000355C5276780000031
:1048E000130101FF23261100EFE05FC9130530001B
:1048F000EF00107B8320C1001301010167800000DD
:10490000130101FF23261100EFE01FC6130530003D
:10491000EF0010798320C1001301010167800000BE
:10492000130101FF2326110023248100232291007B
:10493000130405002328C54293048500138605004F
:1049400093850400EFE04FDC138604000325040088
:1049500083254400EFE04FF513050400EFF05FFA04
:1049600013050400EFE0DF9E13050400EFF05FF78E
:10497000930710002303F40C8320C100032481005B
:10498000832441001301010167800000130510001A
:10499000678000008327454183C707002310F60086
:1049A00003254541678000008327854183C7270091
:1049B0002310F60003258541678000008327C54149
:1049C00083C727002310F6000325C5416780000038
:1049D0008327054293952500B387B70003A50700F9
:1049E000834705002310F6006780000003C74500D9
:1049F00083C7550093978700B3E7E70013F6F70FD7
:104A000003C7050013773700930610006306D70A23
:104A10009316870193D68641638A06009306200089
:104A2000630ED70C13051000678000008347650CE8
:104A300093F7F70F13072000638EE7008347650C99
:104A400093F7F70F130730006386E7001305100094
:104A5000678000008347054163840704B70700208F
:104A6000130710002386E768834725416380070406
:104A7000B70700209387C76803C70700136727009D
:104A80002380E700B70700209387C7682328F50C29
:104A900093072000232EF50C13050000678000000B
:104AA000B7070020238607686FF01FFCB7070020B8
:104AB000238607686FF01FFD8347650C93F7F70F98
:104AC000130730006386E7001305100067800000BD
:104AD0009307100063F6C7001305100067800000FD
:104AE000B70700209387C7682328F50C9307200099
:104AF000232EF50C13050000678000000347650CAA
:104B00001377F70F930630006306D70013051000E4
:104B1000678000009397870193D7874163CE070290
:104B2000931736003386C74093172600B307F50066
:104B300003C7E726B70700202386E768B7070020EA
:104B40009387C7682328F50C93072000232EF50CC4
:104B500013050000678000001376F60793173600F0
:104B60003386C74093172600B307F50003C7A70C89
:104B7000B70700202386E7686FF05FFC130101FF91
:104B80002326110023248100232291009304050091
:104B90001384050083C7050093F737006388070275
:104BA00013071000638AE71003A5C40D63040514FE
:104BB000034764008347740093978700B3E7E700D7
:104BC00063940710130510006F00001383C72500BE
:104BD00083C5350093958500B3E5F50093D785002F
:104BE00093F5F50F13072000638CE7066372F70255
:104BF00013073000638AE7081307F000E396E7FA2B
:104C00001306C50DEFF09FDB23A8A40C6FF0DFF9AE
:104C100013071000E39AE7F89387F7FF93972700AD
:104C20003707000813074729B307F70083A70700D2
:104C30001306C50DE780070023A8A40C03476400F2
:104C40008347740093978700B3E7E70013070004D6
:104C5000E39CE7F49307800023AEF40C6FF0DFF4DD
:104C60009387F7FF93972700370700081307472913
:104C7000B307F70083A707001306C50DE7800700F9
:104C800023A8A40C6FF05FF213075000E36EB7F097
:104C90009387F7FF939727003707000813074729E3
:104CA000B307F70083A707001306C50DE7800700C9
:104CB00023A8A40C6FF05FEF8327054383A7C700E9
:104CC000E78007006F0040036370F50283D5C40CD2
:104CD000636EB500EF501052631A05009307100081
:104CE000A386F4426F00800023AEF40C130500008D
:104CF0006F008000130510008320C1000324810091
:104D000083244100130101016780000013050000A6
:104D1000678000008347650C93F7F70F13072000A7
:104D2000638AE70013073000638AE7021305100067
:104D3000678000008347450C638607001305100059
:104D4000678000009307450C2328F50C930710009B
:104D5000232EF50C13050000678000008347450CE7
:104D60006396070013051000678000009307450C49
:104D70002328F50C93071000232EF50C13050000D3
:104D80006780000083C52500B7070020A384B768AB
:104D90009307100063F6B70013051000678000004A
:104DA000130101FF232611002324810013040500B1
:104DB0008347650C93F7F70F130720006380E70222
:104DC000130730006382E704130510008320C1003D
:104DD0000324810013010101678000006382050242
:104DE0008327054383A74700E7800700B707002014
:104DF00083C797682302F40C930730002303F40C55
:104E0000130500006FF09FFC63960502832705439E
:104E100083A78700E7800700B707002083C797684C
:104E20002302F40C930720002303F40C1305000065
:104E30006FF0DFF98347450CE38AF5FE83270543CE
:104E400083A78700E7800700B707002083C597681E
:104E50002302B40C8327044383A7470013050400EF
:104E6000E78007006FF09FFC8347650C93F7F70F0F
:104E7000130730006386E700130510006780000009
:104E800003C745009307100063F6E7001305100001
:104E90006780000083270543938717002328F50CBC
:104EA00093071000232EF50C130500006780000007
:104EB0008347650C93F7F70F130730006386E7000D
:104EC000130510006780000003C74500930710001A
:104ED00063F6E700130510006780000003C7250094
:104EE00083270543A380E7001305000067800000C7
:104EF000130500006780000003C7450083C7550005
:104F000093978700B3E7E7006390070803C765003E
:104F100083C7750093978700B3E7E700639A070696
:104F200083C5250093F5F507A302B50C8347650CEF
:104F300093F7F70F130730006396E700130510008F
:104F400067800000130101FF232611002324810044
:104F500013040500EFF0DF958347540C63800702CC
:104F6000930720002303F40C130500008320C100E5
:104F700003248100130101016780000093071000E2
:104F80002303F40C6FF05FFE130510006780000030
:104F9000130510006780000083C7050093F73700F2
:104FA000638A0700130720006380E70613051000DB
:104FB000678000008347650C93F7F70F1307200005
:104FC000638EE7008347650C93F7F70F13073000F4
:104FD0006386E700130510006780000003C7250003
:104FE00083C7350093978700B3E7E70013071000E6
:104FF0006386E70013050000678000009307100038
:105000002309F5406FF01FFF83C645008347650CF9
:1050100093F7F70F130730006386E70013051000BE
:105020006780000003C7250083C73500939787007A
:10503000B3E7E7006398070063860600930700085C
:105040006396F6001305000067800000130101FF5E
:105050002326110093850600EFF0CFF8130500001A
:105060008320C100130101016780000083C7050090
:1050700093F73700638A0700130720006380E70671
:1050800013051000678000008347650C93F7F70F46
:1050900013072000638EE7008347650C93F7F70F33
:1050A000130730006386E7001305100067800000D7
:1050B00003C7250083C7350093978700B3E7E70050
:1050C000130710006386E7001305100067800000D7
:1050D00023090540130500006780000083C64500D2
:1050E0008347650C93F7F70F130730006386E700DB
:1050F000130510006780000003C7250083C7350033
:1051000093978700B3E7E70063980700638606007C
:10511000930700086396F6001305000067800000FF
:10512000130101FF23261100232481002322910073
:10513000138405009304050093850600EFF00FF13A
:1051400083A7044383A7C7009305040013850400C5
:10515000E7800700130500008320C10003248100BD
:10516000832441001301010167800000130101FF46
:105170002326110083C7150013972700B7070008DF
:1051800093870726B387E70083A70700E780070018
:105190008320C10013010101678000008347650C73
:1051A00093F7F70F130730006386E700130510002D
:1051B0006780000003C745009307100063F6E7000F
:1051C0001305100067800000130101FF2326110062
:1051D0008327054383A7C700E78007008320C1001A
:1051E00013010101678000001305000067800000C3
:1051F000130101FF2326110023248100130405005D
:1052000093050008EFF00FDE93050000130504007E
:10521000EFF04FDD13050400EFE01F9B8320C1007A
:10522000032481001301010167800000130101FFC5
:105230002326110023248100130405008356C50D85
:105240000326050D93050000EFF08FD20327C40D50
:105250008357C40C63F0E702930710002306F4425F
:10526000130500008320C100032481001301010104
:1052700067800000930720002306F4426FF05FFE72
:10528000130101FF232611002324810013040500CC
:10529000835605280326452793050000EFF00FC627
:1052A000032704288357042763F0E702930730009D
:1052B0002306F442130500008320C100032481006B
:1052C0001301010167800000930740002306F442A8
:1052D0006FF05FFE130101FF2326110023248100DC
:1052E00013040500930750002306F54293060000BF
:1052F0001306000093050000EFF08FC713050400AC
:10530000EFE09F8C130500008320C100032481007F
:105310001301010167800000130101FF2326110022
:105320002324810013040500930760002306F5423F
:10533000930600001306000093050000EFF00FBC79
:1053400013050400EFE05F88130500008320C1000F
:10535000032481001301010167800000130101FE95
:10536000232E1100232C81001304050083274542BE
:105370002324F100032785422326E10093F7070643
:1053800013070002638CE70413070004638EE7042D
:10539000638207029305810013050400EFF05FE5C7
:1053A000130500008320C1010324810113010102C0
:1053B0006780000093058100EFF05FDBE31C05FCD4
:1053C0008357E100638807028307810063CA0702ED
:1053D00013050400EFF0DFEA6FF09FFC93058100F6
:1053E000EFF0DFDB6FF09FFD93058100EFF0DFDF73
:1053F0006FF0DFFC13050400EFF0DFED6FF05FFAF4
:1054000013050400EFF09FE26FF09FF9130101FD17
:10541000232611022324810213040103232EA4FC5A
:1054200093870500A30DF4FC8347B4FD6392070A3C
:105430008327C4FD9387C7262326F4FE8327C4FD54
:1054400083C7C742130730006388E7001307400093
:105450006388E7026F00C00B8327C4FE83A7470160
:105460000327C4FE035747003387E7408327C4FE62
:1054700023AAE7000325C4FDEFF09FE06F00400979
:105480008327C4FD83C7670C13F7F70F930730001A
:105490006316F7028327C4FD83A7074383A7470149
:1054A000638E07008327C4FD83A7074383A74701B3
:1054B000930500000325C4FDE78007008327C4FE91
:1054C00023AA07000325C4FDEFF0DFE06F004004CE
:1054D0008327C4FD83A7074383A74701638A070285
:1054E0008327C4FD83C7670C13F7F70F93073000BA
:1054F0006310F7028327C4FD83A7074303A747016F
:105500008347B4FD938507000325C4FDE70007002A
:1055100093070000138507008320C1020324810242
:105520001301010367800000130101FD232611020E
:105530002324810213040103232EA4FC9387050076
:10554000A30DF4FC8347B4FD6398070C8327C4FDC7
:105550009387870C2326F4FE8327C4FD83C7C742A5
:10556000130710006388E700130720006388E70231
:105570006F00800E8327C4FE83A747010327C4FE64
:10558000035747003387E7408327C4FE23AAE70079
:105590000325C4FDEFF09FC96F00000C8327C4FDF5
:1055A00083C7D742638207029306000013060000F8
:1055B000930500000325C4FDEFF08F9B8327C4FDF6
:1055C000A38607426F0040098327C4FD83C7670C89
:1055D00013F7F70F930730006316F7028327C4FD14
:1055E00083A7074383A70701638E07008327C4FDB2
:1055F00083A7074383A70701930500000325C4FD84
:10560000E78007008327C4FE23AA07000325C4FD03
:10561000EFF09FD06F0040048327C4FD83C7670C61
:1056200013F7F70F930730006318F7028327C4FDC1
:1056300083A7074383A70701638007028327C4FD6D
:1056400083A7074303A707018347B4FD938507009A
:105650000325C4FDE700070093070000138507003A
:105660008320C1020324810213010103678000002B
:10567000130101FE232E1100232C810013040500C9
:1056800013051070EFD04F95370500401305054006
:10569000EFD08FBF93072000630CF4069307100030
:1056A000630EF40683A741732310F1002311010058
:1056B00023120100231601002307010093050100B6
:1056C0003704004013050440EFD08FCB130504408E
:1056D000EFD04FDC9305100013050440EFD04FDFEF
:1056E0009305100013050440EFD04FE1930500002F
:1056F00013050440EFD00FDB13050440EFD08FD724
:105700008320C1010324810113010102678000008D
:105710009307B0002324F1006FF0DFF8B7370000E3
:105720009387F7ED2324F1006FF0DFF7130101FFFA
:1057300023261100B707002023A8A76813850500BA
:10574000EFF01FF3B707002083A70769E39C07FE6C
:105750003705004013050540EFD0CFD28320C100AC
:105760001301010167800000130101FF23261100CE
:1057700013050000EFD04F8FB777DC02938707C087
:10578000630AF502B7A74A0493870720630EF5045E
:10579000B7E7B805938707806318F502B7070020BD
:1057A0003707C00023AAE7681307700023AAE17235
:1057B0006F008001B70700203707400023AAE76881
:1057C0001307300023AAE172B707002003A5476939
:1057D000EFD08F871305C050EFD00F808320C1001A
:1057E0001301010167800000B707002023AA0768A2
:1057F0001307500023AAE1726FF01FFD130101FF90
:105800002326110013060000930510001305600500
:10581000EFD0CFD11305C071EFC01FFC37050400D6
:10582000EFD08FE513060000930500003705040054
:10583000EFD00FD537050400EFD0CFE213060000FC
:10584000930530001305D003EFD04FCE8320C10065
:105850001301010167800000130101FF23261100DD
:1058600013051070EFC05FF71306000093052000CA
:1058700013050003EFD08FCB8320C100130101017A
:1058800067800000130101FF23261100930520000B
:10589000EFF0DFE98320C100130101016780000000
:1058A000130101FF2326110093051000EFF01FE8FC
:1058B0008320C1001301010167800000130101FF73
:1058C00023261100930510003705004013050540FD
:1058D000EFD00FC1631805008320C100130101013F
:1058E0006780000093051000370500401305054050
:1058F000EFD0CFC0B707002083A70769638E0700EA
:10590000B70700209387076903A707001307F7FF6E
:1059100023A0E7006FF05FFC37050040130505404A
:10592000EFD04FB66FF05FFB130101FF232611008C
:105930003705002013058506EFE00FB08320C10076
:10594000130101016780000067800000130101FF5F
:1059500023261100B70700209387870683C77700A7
:10596000639C070037050400EFD00FD18320C100EE
:105970001301010167800000EFC05FCAB707002074
:1059800003A54769EFC05FEC1305C050EFC0DFE42B
:105990003705002013058506EFE04FA76FF09FFC49
:1059A000130101FF23261100EFF05FF18320C100F6
:1059B0001301010167800000130101FF232611007C
:1059C0002324810023229100930405003704002042
:1059D000130404009305C403EFE05FBE9305540372
:1059E00013850400EFE09FBD930554021385040066
:1059F000EFE0DFBC130500008320C1000324810019
:105A0000832441001301010167800000130101FF9D
:105A10002326110023248100130405009305100898
:105A2000EFE0DFC79305300013050400EFE01FC768
:105A30009305200813050400EFE05FC6130500007E
:105A40008320C1000324810013010101678000004D
:105A5000130101FF23261100638E05009307300018
:105A60006380F502130520008320C10013010101AA
:105A700067800000EF004016130520006FF0DFFE86
:105A8000130710002388E18093053000EFE0DFE387
:105A9000B707002023ACA768130500006FF0DFFCF8
:105AA000930710006386F50013052000678000004F
:105AB000130101FF232611002324810023229100DA
:105AC00023202101138405009304050093F6F507B4
:105AD000939736003386D740131726001306070026
:105AE0003307E5000329470D3307C5008355C70C6D
:105AF00013050900EF4010706314050063140902D8
:105B000013071000A388E180130500008320C10063
:105B100003248100832441000329010013010101B2
:105B20006780000093060000130600009305040040
:105B300013850400EFE0DFC36FF01FFD83C715007E
:105B400013070002638AE700130710026388E70265
:105B5000130500006780000023A2F18093878177FE
:105B6000232AF52603C7650083C77500939787002E
:105B7000B3E7E7002320F5286FF09FFD13878180AE
:105B800083260700238CD17613D6860093878177EE
:105B9000A380C70013D606012381C70093D68601D0
:105BA000A381D700834647002382D700834657004E
:105BB000A382D700034767002383E7002328F50C5F
:105BC00003C7650083C7750093978700B3E7E700B5
:105BD000232EF50C6FF0DFF703A741809307F00F3A
:105BE000630CF70403C781779387817783C6170017
:105BF000939686003367D70083C6270093960601E5
:105C00003367D70083C63700939686013367D70082
:105C10009386818023A0E60003C747002382E60025
:105C200003C75700A382E60083C767002383F600FB
:105C30001307F00F23A2E180130500006780000026
:105C4000130101FF2326110093870184239007008D
:105C500023910700EFD04F8B13052000EFD04F8B1F
:105C6000EFF09FB0EFF05FBFEFF05FB937060020B5
:105C7000130646049305100037050020130585061A
:105C8000EFE01FCA8320C1001301010167800000FB
:105C9000130101FF2326110083D70184130790030A
:105CA000638AE7066372F7061307F0036382E7046B
:105CB000130710046390E708B707002083A58769DE
:105CC0001385C184EF30C03E630A05062388018036
:105CD000930600041386C184930530003705002025
:105CE00013058506EFE09FA11307F0032390E184DD
:105CF00003C70181930710006318F704130710040A
:105D00002390E1846FF05FFB639607021307900313
:105D10002390E184B70700209387870683C7670C29
:105D200093F7F70F13073000E382E7FA130500003B
:105D30006F00C00023900184130530008320C10050
:105D40001301010167800000130500006FF01FFFC1
:105D5000130101FF2326110023248100938701846E
:105D600083D727001307C0046384E704637AF7022C
:105D70001307F0046380E706130740056390E70A02
:105D800003C71181930710006306F708130500008D
:105D90008320C100032481001301010167800000FA
:105DA000639E0706938701841307C0042391E700CD
:105DB000B70700209387870683C7670C93F7F70F11
:105DC000130730006394E706938701841307F004F8
:105DD0002391E7001384018413058400EF3000460B
:105DE0002322A40063080504A3880180138401848E
:105DF000835684001306050093051008370500201C
:105E000013058506EFE0DF96930740052311F400A4
:105E10006FF01FF7EF3040456FF01FFB9387018451
:105E200023910700130530006FF09FF61305000063
:105E30006FF01FF6130500006FF09FF5130101FFCF
:105E4000232611002324810013052060EFC0DF9872
:105E5000930620001306200093050001371401402B
:105E600013050480EFC01F859305200013050480EF
:105E7000EFC05F949306000813062000930500010D
:105E800013050480EFC01F839305000813050480E9
:105E9000EFC05F928320C100032481001301010140
:105EA00067800000130101FF232611006300050233
:105EB000930520003715014013050580EFC01F8FA3
:105EC0008320C100130101016780000093052000B9
:105ED0003715014013050580EFC0DF8D6FF05FFEC1
:105EE000130101FF232611002324810013053060D4
:105EF000EFC09F8EB7260000130610009305000127
:105F000037140140130504C0EFC0CFFAB7460000B4
:105F10001306100093050001130504C0EFC08FF9AC
:105F2000B78600001306100093050001130504C096
:105F3000EFC04FF8B7160000130600009305800469
:105F4000130504C0EFC00FF79306100013061000EE
:105F500093054001130504C0EFC0CFF58320C100B5
:105F6000032481001301010167800000130101FF78
:105F70002326110023248100B72600001306000009
:105F80009305000037140140130504C0EFC08FF2E1
:105F9000B74600001306000093050000130504C077
:105FA000EFC04FF1B7860000130600009305000014
:105FB000130504C0EFC00FF0B71600001306000071
:105FC00093050000130504C0EFC0CFEE9306100048
:105FD0001306000093050000130504C0EFC08FED09
:105FE0008320C100032481001301010167800000A8
:105FF000130101FF2326110063000502B7450000CD
:1060000037150140130505C0EFC04FFA8320C100CA
:106010001301010167800000B745000037150140FA
:10602000130505C0EFC00FF96FF05FFE130101FF0C
:106030002326110063000502B785000037150140D3
:10604000130505C0EFC08FF68320C10013010101C5
:1060500067800000B785000037150140130505C0B3
:10606000EFC04FF56FF05FFE130101FF2326110013
:1060700063000502B725000037150140130505C070
:10608000EFC0CFF28320C10013010101678000003F
:10609000B725000037150140130505C0EFC08FF18B
:1060A0006FF05FFEF32600B0F32700B0B387D74050
:1060B00013073006E37AF7FE67800000130101FF43
:1060C00023261100B715000037150140130505C040
:1060D000EFC0CFEE630A0500130510008320C10056
:1060E0001301010167800000130500006FF01FFF1E
:1060F000130101FF23261100630005029305100020
:1061000037150140130505C0EFC04FEA8320C100D9
:10611000130101016780000093051000371501404D
:10612000130505C0EFC00FE96FF05FFEF32600B066
:10613000931715003385A70013175500F32700B0F8
:10614000B387D740E3ECE7FE67800000130101FF4F
:1061500023261100EFF0DFD813051000EFF05FE900
:1061600013051000EFF09FEC13050000EFF0DFEFD8
:10617000B707002023AE07688320C1001301010187
:1061800067800000130101FF23261100EFF01FDEDE
:106190008320C1001301010167800000B7070020C0
:1061A0009387C76983A607001307F0006360D720B1
:1061B000939726003707000813078734B387E70053
:1061C00083A707006780070063180500B707002052
:1061D0001307100023AEE768B707002003A5C769BF
:1061E00067800000E30A05FEB707002013072000C0
:1061F00023AEE7686FF05FFE630A0500B707002073
:106200001307300023AEE7686FF01FFDB7070020CB
:106210001307400023AEE7686FF01FFC630805001A
:10622000B707002023AE07686FF01FFBB7070020F9
:106230001307A00023AEE7686FF01FFA630A05009A
:10624000B70700201307600023AEE7686FF0DFF8A0
:10625000B70700201307500023AEE7686FF0DFF7A1
:10626000E30C05F6B70700201307600023AEE768CC
:106270006FF09FF6630A0500B70700201307900030
:1062800023AEE7686FF05FF5B707002013077000D3
:1062900023AEE7686FF05FF4E30005F4B707002072
:1062A0001307800023AEE7686FF01FF3630A050051
:1062B000B70700201307900023AEE7686FF0DFF107
:1062C000B70700201307500023AEE7686FF0DFF038
:1062D000630A0500B70700201307200023AEE76814
:1062E0006FF09FEFB70700201307100023AEE76899
:1062F0006FF09FEE630A0500B70700201307C00088
:1063000023AEE7686FF05FEDB70700201307B0001A
:1063100023AEE7686FF05FECE30005ECB707002001
:106320001307C00023AEE7686FF01FEB630A050098
:10633000B70700201307F00023AEE7686FF0DFE92E
:10634000B70700201307D00023AEE7686FF0DFE83F
:10635000E30405E8B70700201307E00023AEE76871
:106360006FF09FE7630A0500B70700201307F000EE
:1063700023AEE7686FF05FE6B70700201307B000B1
:1063800023AEE7686FF05FE5630A0500B7070020FA
:106390001307200023AEE7686FF01FE4B707002063
:1063A0001307100023AEE7686FF01FE36F000000D3
:1063B000130101FF232611002324810023229100D1
:1063C0009304050013840500EFF09FC21305040039
:1063D000EFF0DFC5EFF01FCD13051000EFF0DFC8C1
:1063E000EFF0DFCD13040500EFF0DFCB1305000065
:1063F000EFF09FC713850400EFF05FDA1305040088
:106400008320C10003248100832441001301010182
:1064100067800000B707002083A7C7699387E7FF5D
:10642000130810006374F8006F0000006308050093
:1064300063880500631806006F0000006F0000000D
:106440006F000000130101FE232E1100232C810098
:10645000232A9100232821012326310123244101ED
:1064600023225101232061011309070093840600B0
:10647000130A0600138B050093090500930510000D
:1064800013050000EFF0DFF2930510001305000084
:10649000EFF01FF2130400006F004001930510009D
:1064A00013050000EFF0DFF013041400E36894FE1E
:1064B000930400006F00C00213050000EFF05FEFCF
:1064C000630C05043384890093071000B39A5701C5
:1064D00083270400B3E757012320F40093841400BA
:1064E00063FC440513D4540013142400B3078B0039
:1064F00083A5070093FAF401B3D5550193F5150070
:106500009307FAFFE39A97FAE31809FA13051000C4
:10651000EFF01FEA6FF0DFFA338489009307100071
:10652000B397570193C7F7FF03270400B377F7002A
:106530002320F4006FF09FFA130400006F00400165
:106540009305100013051000EFF09FE613041400EC
:10655000637E24019307F9FFE38487FE930510000F
:1065600013050000EFF0DFE46FF05FFE930510000D
:1065700013051000EFF0DFE3930510001305000092
:10658000EFF01FE3B707002003A7C76993071000C8
:106590006304F7006F0000008320C1010324810120
:1065A00083244101032901018329C100032A8100B9
:1065B000832A4100032B01001301010267800000C0
:1065C000B707002003A7C769930710006304F7000B
:1065D0006F000000130101FF232611002324810016
:1065E0002322910023202101130906009384050032
:1065F000130405009305100013051000EFF05FDB96
:106600001307100093060000130609009385040089
:1066100013050400EFF01FE08320C1000324810074
:106620008324410003290100130101016780000058
:10663000B707002003A7C769930710006304F7009A
:106640006F000000130101FF2326110023248100A5
:1066500023229100232021011309060093840500C1
:10666000130405009305100013051000EFF05FD42C
:106670009305100013051000EFF09FD3130750008F
:106680009306000013060900938504001305040017
:10669000EFF05FD88320C1000324810083244100F0
:1066A000032901001301010167800000130101FFAC
:1066B0002326110023248100130400006F004001F1
:1066C0009305100013051000EFF09FCE1304140083
:1066D00093075000E3D687FE9305100013050000D2
:1066E000EFF01FCDB707002003A7C769930710007D
:1066F0006304F7006F0000008320C10003248100C1
:106700001301010167800000B707002003A7C769D4
:10671000930710006308F7026F0000009305100054
:1067200013050000EFF0DFC813041400E36894FEC3
:10673000B707002003A7C769930710006302F70299
:106740006F000000130101FF2326110023248100A4
:106750002322910093040500130400006FF01FFD35
:106760008320C1000324810083244100130101011F
:106770006780000037050008130585386780000032
:10678000371500001305C57167800000130101FF74
:106790002326110023248100130405009387C18858
:1067A00083D727001307E019638CE7066370F704AB
:1067B0001307201A6386E70A1307501A6394E70C3D
:1067C0009385C188138645109385450113054000C4
:1067D000EF10D07A9307100063F6A7109387C18853
:1067E00083A747012320F4006F00C009638A070ACA
:1067F0001307C0196398E7089387C1881386471069
:1068000083A5070613057001EF20000F9307100002
:1068100063FEA70A9387C1881307E0192391E70055
:106820009385C188138645109385C50513056001BE
:10683000EF10D0749307100063FEA7089387C188F8
:1068400083A7C70593F70770638A07069387C188F4
:106850001307007023AEE7041307201A2391E70003
:106860009387C1881386471083A5C7051305600168
:10687000EF2080089307100063F2A7069307F0FF4C
:106880002320F4009387C18823910700130530006B
:106890008320C100032481001301010167800000EF
:1068A0009387C1883707220023A0E7062390B70605
:1068B0001307C0192391E7006FF01FF49387C18875
:1068C0001307501A2391E7006FF09FEF13050000A4
:1068D0006FF01FFC130500006FF09FFB1305000015
:1068E0006FF01FFB130500006FF09FFA130101FF0B
:1068F0002326110023248100130405009387C188F7
:1069000083D727001307B020638CE708637CF70266
:10691000130710216388E70E130740216386E712EF
:106920001307D0206380E70A9387C188239107006B
:10693000130530008320C1000324810013010101ED
:10694000678000006384070E13075020E39EE7FC76
:106950009387C1881386471083A5870113055000CC
:10696000EF1090799307100063F6A7109387C18802
:1069700023A0070613072000A381E70603A7070645
:10698000B70690FF9386F6FF3377D700B70620004F
:106990003367D70023A0E7061307B0202390E70052
:1069A0009387C1881386471083A5070613057001D6
:1069B000EF1090749307100063F2A70C1307D02018
:1069C0002396E1889385C188138645109385C50574
:1069D00013056001EF10905A9307100063F4A70AA3
:1069E0009387C18883A7C70593F70770638A070455
:1069F0009387C1881307007023AEE70413071021A3
:106A00002390E7009387C1881386471083A5C705A5
:106A100013056001EF10506E9307100063F8A7068E
:106A20009307F0FF2320F4006FF01FF09387C188D5
:106A300023ACB700130750202390E7006FF05FF1FD
:106A4000130740212396E1889385C188138645105A
:106A50009385450113054000EF1050529307100035
:106A600063FAA7029387C18883A747012320F40014
:106A70006FF09FEB130500006FF0DFEB13050000D4
:106A80006FF05FEB130500006FF0DFEA1305000005
:106A90006FF05FEA130500006FF0DFE9130101FFFB
:106AA0002326110023248100130405009387C18845
:106AB00083D727001307F01E638CE708637CF70277
:106AC0001307501F6388E70E1307801F6386E712C2
:106AD0001307101F6380E70A9387C188239107007B
:106AE000130530008320C10003248100130101013C
:106AF000678000006384070E1307901EE39EE7FC87
:106B00009387C1881386471083A58701130550001A
:106B1000EF10905E9307100063F6A7109387C1886B
:106B200023A0070613072000A381E70603A7070693
:106B3000B70690FF9386F6FF3377D700B7061000AD
:106B40003367D70023A0E7061307F01E2390E70062
:106B50009387C1881386471083A507061305700124
:106B6000EF1090599307100063F2A70C1307101F42
:106B70002396E1889385C188138645109385C505C2
:106B800013056001EF10903F9307100063F4A70A0C
:106B90009387C18883A7C70593F70770638A0704A3
:106BA0009387C1881307007023AEE7041307501FB3
:106BB0002390E7009387C1881386471083A5C705F4
:106BC00013056001EF1050539307100063F8A706F8
:106BD0009307F0FF2310F4006FF01FF09387C18834
:106BE00023ACB7001307901E2390E7006FF05FF10E
:106BF0001307801F2396E1889385C188138645106B
:106C00009385450113054000EF105037930710009E
:106C100063FAA7029387C18883A747012310F40072
:106C20006FF09FEB130500006FF0DFEB1305000022
:106C30006FF05FEB130500006FF0DFEA1305000053
:106C40006FF05FEA130500006FF0DFE9130101FF49
:106C50002326110023248100130405009387C18893
:106C600083D727001307301D6388E708637CF7028A
:106C70001307901D6384E70E1307C01D6382E7129C
:106C80001307501D638CE7089387C1882391070081
:106C9000130530008320C10003248100130101018A
:106CA000678000006380070E1307D01CE39EE7FC9B
:106CB0009387C1881386471083A587011305500069
:106CC000EF1090439307100063F2A7109387C188D9
:106CD00023A0070613072000A381E70603A70706E2
:106CE000B70690FF9386F6FF3377D70023A0E70619
:106CF0001307301D2390E7009387C1881386471040
:106D000083A5070613057001EF10103F93071000CD
:106D100063F2A70C1307501D2396E1889385C18861
:106D2000138645109385C50513056001EF101025E6
:106D30009307100063F4A70A9387C18883A7C70548
:106D400093F70770638A07049387C188130700705D
:106D500023AEE7041307901D2390E7009387C188B3
:106D60001386471083A5C70513056001EF10D038BF
:106D70009307100063F8A7069307F0FF2300F400C1
:106D80006FF09FF09387C18823ACB7001307D01C26
:106D90002390E7006FF0DFF11307C01D2396E18811
:106DA0009385C188138645109385450113054000DE
:106DB000EF10D01C9307100063FAA7029387C188D5
:106DC00083A747012300F4006FF01FEC13050000B8
:106DD0006FF05FEC130500006FF0DFEB13050000B0
:106DE0006FF05FEB130500006FF0DFEA13050000A2
:106DF0006FF05FEA130101FF2326110023248100B5
:106E00009387C18883D7270013079025638CE706F3
:106E100013040500637CF702130720266382E70E44
:106E200013076026638EE710130700266388E70ABE
:106E30009387C18823910700130530008320C10088
:106E4000032481001301010167800000638C071097
:106E500013077025E39EE7FC9387C18813864710CC
:106E600083A5870113055000EF1010299307100028
:106E700063F4A7109387C18823AA8700130790257E
:106E80002390E7009387C1881386471083A54701A5
:106E900013054000EF1050269307100063F2A70E71
:106EA0009387C18823A0070613072000A381E70664
:106EB00003A70706B70690FF9386F6FF3377D70040
:106EC000B70620003367D700B70601003367D70045
:106ED00023A0E706130700262390E7009387C188C5
:106EE0001386471083A5070613057001EF10D02005
:106EF0009307100063FAA708130720262396E1885A
:106F00009385C188138645109385C50513056001D7
:106F1000EF10D0069307100063FCA7069387C18883
:106F200083A7C70593F70770E38407F09387C188A9
:106F30001307007023AEE704130760262390E700D1
:106F40009387C1881386471083A5C7051305600181
:106F5000EF10901A93071000E3ECA7EC1305000064
:106F60006FF0DFED9387C18823ACB700130770255E
:106F70002390E7006FF05FEE130500006FF01FEC49
:106F8000130500006FF09FEB130500006FF01FEB7F
:106F9000130500006FF09FEA130101FF2326110083
:106FA000232481009387C18883D727001307E02318
:106FB000638CE70613040500637CF7021307702453
:106FC0006382E70E1307B024638EE7101307502483
:106FD0006388E70A9387C18823910700130530006F
:106FE0008320C10003248100130101016780000098
:106FF000638C07101307C023E39EE7FC9387C188C7
:107000001386471083A5870113055000EF10D00E9B
:107010009307100063F4A7109387C18823AA870001
:107020001307E0232390E7009387C1881386471056
:1070300083A5470113054000EF10100C93071000C3
:1070400063F2A70E9387C18823A0070613072000C9
:10705000A381E70603A70706B70690FF9386F6FF0E
:107060003377D700B70610003367D700B7060100A3
:107070003367D70023A0E706130750242390E700C7
:107080009387C1881386471083A5070613057001EF
:10709000EF1090069307100063FAA70813077024F7
:1070A0002396E1889385C188138645109385C5058D
:1070B00013056001EF10806C9307100063FCA706B6
:1070C0009387C18883A7C70593F70770E38407F008
:1070D0009387C1881307007023AEE7041307B02419
:1070E0002390E7009387C1881386471083A5C705BF
:1070F00013056001EF10500093071000E3ECA7ECBC
:10710000130500006FF0DFED9387C18823ACB70053
:107110001307C0232390E7006FF05FEE1305000014
:107120006FF01FEC130500006FF09FEB13050000DC
:107130006FF01FEB130500006FF09FEA130101FFD2
:1071400023261100232481009387C18883D7270039
:1071500013073022638CE70613040500637CF702F3
:107160001307C022638EE70C13070023638AE7101E
:107170001307A0226384E70A9387C188239107003D
:10718000130530008320C100032481001301010195
:10719000678000006388071013071022E39EE7FC56
:1071A0009387C1881386471083A587011305500074
:1071B000EF1080749307100063F0A7109387C188C5
:1071C00023AA8700130730222390E7009387C18802
:1071D0001386471083A5470113054000EF10C071C7
:1071E0009307100063FEA70C9387C18823A00706AE
:1071F00013072000A381E70603A70706B70690FF41
:107200009386F6FF3377D700B70601003367D700C0
:1072100023A0E7061307A0222390E7009387C188E5
:107220001386471083A5070613057001EF10C06C85
:107230009307100063FAA7081307C0222396E1887A
:107240009385C188138645109385C5051305600194
:10725000EF10C0529307100063FCA7069387C18804
:1072600083A7C70593F70770E38807F09387C18862
:107270001307007023AEE704130700232390E700F1
:107280009387C1881386471083A5C705130560013E
:10729000EF10806693071000E3E0A7EE13050000EF
:1072A0006FF05FEE9387C18823ACB70013071022FD
:1072B0002390E7006FF0DFEE130500006FF09FEC06
:1072C000130500006FF01FEC130500006FF09FEB3B
:1072D000130500006FF01FEB130101FF23261100BF
:1072E000232481009387C18883D727001307901B2D
:1072F000638AE708138405006376F7041307B01B5D
:107300006386E70A1307F01B6390E7029387C1883F
:107310001386471083A5C70513056001EF10C05DF4
:107320009307100063FAA70E9387C1882391070083
:10733000130530008320C1000324810013010101E3
:10734000678000006386070A1307101BE39EE7FCB3
:107350001386C188130646109305050013054000E7
:10736000EF1080599307100063FCA7089387C1882A
:107370003707230023A0E706239087061307901BF7
:107380002391E7009387C1881386471083A50706DA
:1073900013057001EF1040569307100063F6A7061F
:1073A0009387C1881307B01B2391E7009385C18899
:1073B000138645109385C50513056001EF10003C49
:1073C0009307100063F6A7049387C18883A7C705B6
:1073D00093F70770E38A07F49387C1881307007057
:1073E00023AEE7041307F01B2391E7006FF01FF2B1
:1073F0009387C1881307101B2391E7006FF05FF597
:10740000130500006FF01FF3130500006FF09FF2EB
:10741000130500006FF01FF2130500006FF09FF1DD
:10742000130101FF232611009387C18823900700D1
:107430002391070023A407109387C18803A787100F
:107440009307300063E6E7029386C188931717001D
:10745000B387E70093972700B387F6001306500021
:1074600023A2C7121307170023A4E6106FF0DFFC56
:10747000EF10802D1385C18813050511EF001077DB
:1074800093071000E3F8A7FE1385C1881305451183
:10749000EF10800B93071000E3F8A7FE9387C188D5
:1074A0001307100023A2E7049387C18813864710AF
:1074B00083A5470413050001EF1000449307100053
:1074C000E3F4A7FE8320C1001301010167800000DF
:1074D000130101FF232611009387C18823A207040B
:1074E0009387C1881386471083A5470413050001BD
:1074F000EF10804093071000E3F4A7FEEF10802602
:107500008320C1001301010167800000130101FF06
:1075100023261100232481001304050083D7C1888A
:10752000130790076382E7041307B0076384E70833
:10753000638E070023960188130530008320C10065
:10754000032481001301010167800000232005004E
:107550009387C1881307100023A4E7106F0000046D
:10756000130790072396E1889387C18883A7871024
:1075700013952700B7150000B385B7003305A400A5
:10758000EFF0CFA09307100063F4A7049387C1889E
:1075900003A787101307170023A4E7109387C18858
:1075A00003A787109307F001E3FCE7FA1307B0077E
:1075B0002396E1889305107B13050408EFF00F9DD7
:1075C00093071000E3E8A7F6130500006FF01FF71C
:1075D000130500006FF09FF6130101FF2326110031
:1075E000232481001304050083D7C1881307800872
:1075F000638EE70A637AF7021307C0086380E70E19
:107600001307E008638AE7101307A008638AE706F8
:1076100023960188130530008320C10003248100D4
:1076200013010101678000006386070213076008E9
:10763000E390E7FEB7170000B385F50013050400DB
:10764000EFF0CF9493071000E3E4A7FC13050000CC
:107650006FF09FFC9307F00163C8B7001307600841
:107660002396E1886FF01FFD93070002638CF502FB
:107670009307000463CAB7041307A0082396E188A0
:10768000B71700009387F7FFB385F50013050400D3
:10769000EFF0CF8F93071000E3ECA7F6130500007F
:1076A0006FF09FF7130780082396E1889305107BFE
:1076B00013050400EFF08F8D93071000E3EAA7F4A1
:1076C000130500006FF05FF5B717000093870704FC
:1076D00063C4B7021307C0082396E1889385F5FBBE
:1076E00013050400EFF08F8A93071000E3E2A7F27E
:1076F000130500006FF05FF2B717000093871704BF
:107700006388F5009307F0FF2320F5006FF05FF02A
:107710001307E0082396E1889305007B1385C18851
:107720001305C510EFF08F869307100063FCA700C8
:107730009387C18883A7C71093F737002320F400ED
:107740006FF01FED130500006FF01FED130101FF37
:1077500023261100232481002322910023202101CC
:1077600013040500938405001309060083D7C1881C
:107770001307E0096386E708637CF7041307200A10
:107780006382E7101307600A6398E70A9387C1884A
:1077900003A58710B30595003305A400EFF00FCBC8
:1077A0009307100063FCA7129387C18803A7871073
:1077B0001307170023A4E7109387C18883A78710B6
:1077C00063FC27071307600A2396E1886FF01FFC0C
:1077D00063940706937735006390070893F73500A5
:1077E000639C070693773600639807069387C188E2
:1077F00023A407106F0080031307E0092396E18894
:107800009387C18803A58710B30595003305A400AD
:10781000EFF0CF8D9307100063FAA70A9387C18812
:1078200003A787101307470023A4E7109387C18895
:1078300083A78710E3E227FD239601881305300014
:107840008320C10003248100832441000329010017
:10785000130101016780000093771400639207060B
:1078600093F71400639E070493771900639A070443
:107870009387C18823A407106F0080031307200A91
:107880002396E1889387C18803A58710B3059500E7
:107890003305A400EFF08FA09307100063FCA7024C
:1078A0009387C18803A787101307270023A4E71035
:1078B0009387C18883A78710E3E227FD6FF0DFF786
:1078C0009387C18823A407106FF01FEF13050000F2
:1078D0006FF01FF7130500006FF09FF6130500000F
:1078E0006FF01FF6130101FF2326110023248100EE
:1078F0002322910023202101130405001389050090
:107900009304060083D7C1881307400B6388E708F8
:10791000637EF7041307800B638CE70E1307C00B1D
:10792000639AE7149387C18883A58710B307B400CF
:10793000B385250103C50700EFF05F8093071000B2
:1079400063F2A7169387C18803A787101307170050
:1079500023A4E7109387C18883A7871063FE970647
:107960001307C00B2396E1886FF0DFFB63940710C9
:10797000937735006398070693F7350063940706FD
:1079800093773600639007069387C18823A4071076
:107990006F00C0031307400B2396E1889387C188CB
:1079A00083A58710B307B400B385250103A507009D
:1079B000EFF04FC49307100063FEA70C9387C188B4
:1079C00003A787101307470023A4E7109387C188F4
:1079D00083A78710E3E097FC9387C18823A407104F
:1079E0006F0080089377140063940706937719005B
:1079F0006390070693F71400639C07049387C1887C
:107A000023A407106F00C0031307800B2396E1889F
:107A10009387C18883A58710B307B400B385250178
:107A200003D50700EFF04FD79307100063F8A706C0
:107A30009387C18803A787101307270023A4E710A3
:107A40009387C18883A78710E3E097FC6FF0DFF886
:107A50009387C18823A407106FF0DFEF9387170087
:107A60001387C1882324F7109387C18883A78710C1
:107A7000E3E697FE23960188130530008320C100BA
:107A80000324810083244100032901001301010123
:107A900067800000130500006FF05FFE1305000013
:107AA0006FF0DFFD130500006FF05FFD130101FFB4
:107AB0002326110083D7C1881307C00D6382E70A0C
:107AC0006372F7041307F00D6386E7121307C00E05
:107AD0006390E7029387C1881386471083A5470404
:107AE00013050001EF0050619307100063F0A71623
:107AF00023960188130530008320C1001301010182
:107B0000678000006386070C1307100DE392E7FE01
:107B10009387C1881386471083A547041305000186
:107B2000EF00905D9307100063F6A71013050000A7
:107B3000EFE00FDC378501001305056AEFE00FDF8A
:107B400013051000EFE0CFDA9387C1883707008074
:107B50001367970023A2E7041307C00D2390E700E3
:107B60009387C1881386471083A547041305000136
:107B7000EF0090589307100063F2A70C9387C18819
:107B800023A407109387C18803A7871093073006A3
:107B900063FEE7049387C1883707008013675700A7
:107BA00023A2E70483A787041397C700635C070039
:107BB0009387C18803A74704B70600103367D7002F
:107BC00023A2E7041307C00E2396E1886FF09FF00D
:107BD0009387C188370700801367B70023A2E704A3
:107BE0001307100D2390E7006FF09FF21307F00DBD
:107BF0002396E1889385C188138645109385850473
:107C000013051001EF0090379307100063FCA702E3
:107C10009387C18883A7870493F70720E39C07F61F
:107C20009387C18803A787101307170023A4E710C1
:107C30006FF05FF5130500006FF01FEC13050000F7
:107C40006FF09FEB130500006FF01FEB13050000B2
:107C50006FF09FEA130101FF2326110083D7C1882B
:107C60001307600F6386E7021307A00F6384E7061C
:107C7000638C070023960188130530008320C10020
:107C800013010101678000001307600F2396E1884C
:107C90009385C1881386451093854504130500011B
:107CA000EF00D02D9307100063F8A7049387C188D5
:107CB00003A74704B70600C09386F6FF3377D700C3
:107CC000B70600803367D70023A2E7041307A00F8D
:107CD0002390E7009387C1881386471083A5470444
:107CE00013050001EF00504193071000E3E4A7F8EB
:107CF000130500006FF09FF8130500006FF01FF8E8
:107D000083D7C188638C070013074010638CE7009A
:107D10002396018813053000678000001307401088
:107D20002396E188130101FF2326110023248100FB
:107D3000130405009385C188138645109385850437
:107D400013051001EF0090239307100063FEA702B4
:107D50009387C18883A7870493F70720638207026C
:107D6000930710002320F4002396018813053000A8
:107D70008320C100032481001301010167800000FA
:107D8000232004006FF05FFE130500006FF05FFE1C
:107D9000130101FF2326110083D7C1881307601147
:107DA0006382E7086372F70413078011638CE708A6
:107DB0001307B0116390E7029387C18813864710B9
:107DC00083A5470413050001EF001033930710004B
:107DD00063F0A70E23960188130530008320C100AD
:107DE00013010101678000006382070A1307401135
:107DF000E392E7FE9305007B1385C1881305C51048
:107E0000EFE0DF989307100063F8A7089387C18815
:107E100003A7C7101377B7FF23A6E7101307601156
:107E20002390E7009305007B9387C18803A5C710C3
:107E3000EFF08FCA9307100063F4A70613078011B1
:107E40002396E1889385C188138645109385450460
:107E500013050001EF0090129307100063F6A704CA
:107E60009387C18803A74704B706008093C6F6FF2F
:107E70003377D700B70600403367D70023A2E70463
:107E80001307B0112390E7006FF01FF313074011A1
:107E90002396E1886FF01FF6130500006FF01FF4C2
:107EA000130500006FF09FF3130500006FF01FF340
:107EB000130500006FF09FF2130101FF232611004C
:107EC00083D7C188130770126382E7086372F704CF
:107ED00013079012638CE7081307C0126390E70240
:107EE0009387C1881386471083A5470413050001B3
:107EF000EF0090209307100063F0A70E23960188EF
:107F0000130530008320C1001301010167800000C8
:107F10006382070A13075012E392E7FE9305007B82
:107F20001385C1881305C510EFE05F869307100025
:107F300063F8A7089387C18803A7C7101367470092
:107F400023A6E710130770122390E7009305007B28
:107F50009387C18803A5C710EFF00FB893071000EF
:107F600063F4A706130790122396E1889385C188CE
:107F7000138645109385450413050001EF0010009A
:107F80009307100063F6A7049387C18803A74704EB
:107F9000B706008093C6F6FF3377D700B7060040D8
:107FA0003367D70023A2E7041307C0122390E7002A
:107FB0006FF01FF3130750122396E1886FF01FF63E
:107FC000130500006FF01FF4130500006FF09FF31E
:107FD000130500006FF01FF3130500006FF09FF210
:107FE000130101FF23261100232481002322910085
:107FF000130405009384060083D7C1881307E01398
:108000006384E706637CF702130760166384E7184E
:1080100013077016638AE71A13075016638CE71468
:1080200023960188130530008320C10003248100BA
:108030008324410013010101678000006380070A67
:108040001307D013E39EE7FC9305007A9387C1885A
:1080500003A58711EFF04FA89307100063FCA71C3E
:108060001307E0132396E1889305107A1385C188DE
:108070001305C511EFE08FF19307100063F0A71C03
:108080001387C1888327C711B7060008B3E7D70055
:10809000B716FFFF9386F6FFB3F7D700B7160000B9
:1080A000B3E7D70093E78704232EF7109307200048
:1080B0006304F41463F0870A930730006308F41430
:1080C000930740006314F40A9387C18803A7C7117C
:1080D0001367370023AEE7106F0040099387C1880C
:1080E00023A407109387C18883A787101307300044
:1080F0006368F70E139717003307F70093162700EE
:108100001387C1883307D70083264712130750000F
:10811000638AE600938717001387C1882324F7102A
:108120006FF05FFC9386C188139717003307F70041
:10813000131727003387E600232287122324B71260
:108140002326C71223ACF6109307D0132390F60012
:108150006FF09FEF93071000631AF4009387C188B4
:1081600003A7C7111367470023AEE7101307501684
:108170002396E1889305107A9387C18803A5C711D8
:10818000EFF08F959307100063FEA70A13076016A0
:108190002396E1889387C18883A6871113971600D9
:1081A0003307D70013172700B387E7009305207A1A
:1081B00003A58712EFF04F929307100063F8A7080A
:1081C000130770162396E1889305107A1385C188EA
:1081D00013050512EFE08FDB9307100063FCA70681
:1081E0009387C18803A7871093074000630AF702AB
:1081F00023A004006FF0DFE29387C18803A7C711B3
:108200001367270023AEE7106FF05FF69387C188EE
:1082100003A7C7111367170023AEE7106FF01FF510
:108220009307E00023A0F4002396018813052000A3
:108230006FF09FDF130500006FF01FDF13050000D4
:108240006FF09FDE130500006FF01FDE13050000C6
:108250006FF09FDD130500006FF01FDD130101FFBC
:1082600023261100232481001384060083D7C188AC
:10827000130780186382E70A13079018638EE70AD2
:10828000638E070023960188130530008320C10008
:108290000324810013010101678000009387C188D6
:1082A00023A407106F000001938717001387C1886C
:1082B0002324F7109387C18883A787101307300002
:1082C0006364F70493961700B386F60013982600AC
:1082D0001387C1883307070103274712E316A7FC5A
:1082E0001387C1883307070103278712E31EB7FAF4
:1082F0001387C188330707010327C712E316C7FA9C
:108300001387C188232CF71013074000638EE706FC
:10831000130780182396E1889305007A9387C18814
:1083200003A58711EFE05FFB9307100063F8A70632
:10833000130790182396E1889305107A130500001F
:10834000EFE09FF99307100063FEA7049387C188AD
:1083500003A6871013171600B305C70093962500D0
:10836000B386D7009305500023A2B61223A40612A9
:108370003307C70093162700B387D70023A6071239
:10838000232004006FF01FF09307E0002320F40087
:1083900023960188130520006FF05FEF130500009E
:1083A0006FF0DFEE130500006FF05FEE130101FFC9
:1083B000232611009387019E23900700238A07003C
:1083C000EFD0DFD8EFE08FAE8320C10013010101B1
:1083D00067800000130101FF23261100EFD09FDA10
:1083E0008320C100130101016780000083D7019E33
:1083F00063920708130101FF232611002324810043
:1084000023229100930405009387019E03C747012F
:10841000930710006310F7041384019E23220400C5
:1084200013060002930544001305C400EFE04F99C2
:108430008327C40023A0F4002390019E130530007D
:108440008320C10003248100832441001301010122
:10845000678000001385019E2322F500230AF500A2
:1084600013065000930545001305C500EFE04F9C2F
:108470006FF09FFA2390019E130530006780000083
:1084800083D7019E63920708130101FF2326110081
:10849000232481009387019E03C7470193070001AE
:1084A0006310F7041384019EB70701002322F40030
:1084B00013060002930544001305C400EFE04F903B
:1084C00003455401631E05022390019E13053000ED
:1084D0008320C10003248100130101016780000093
:1084E0001385019E2322F500230AF5001306500090
:1084F000930545001305C500EFE08F936FF09FFAD9
:10850000EFE08FA06FF05FFC2390019E1305300019
:108510006780000083D7019E638807002390019E37
:108520001305300067800000130101FF23261100AE
:10853000EFE08F9D2390019E130530008320C10042
:10854000130101016780000083D7019E6398070A29
:10855000130101FF2326110023248100232291000F
:10856000930405009387019E03C747019307000109
:108570006316F7061384019E2322040013060002EB
:10858000930544001305C400EFE08F838327C400E4
:1085900023A0F40093D7470093F7F7032301F400D7
:1085A00083A7040093D7C70093F77700A30AF400CA
:1085B000638807009387F7FF1387019EA30AF700DC
:1085C0002390019E130530008320C1000324810005
:1085D0008324410013010101678000001385019E7F
:1085E0002322F500230AF5001306500093054500E9
:1085F0001305C500EFE0CF836FF0DFF72390019EF6
:10860000130530006780000083D7019E639807122E
:108610009387019E03C7270093071000B397E700D5
:108620009387F7FF63F4A7006F000000638C0500D9
:1086300063080600032706009307300063F6E7008F
:108640006F0000006F000000130101FE232E1100D7
:10865000232C8100232A9100232821012326310184
:108660001309060093840500930905009387019E72
:1086700003C7470193071001631EF70883A704008F
:10868000939727000327090013773700B3E7E70024
:108690001384019E2322F40083A7040093D7E701EB
:1086A00013972900B3E7E7002324F40003462400CE
:1086B00013062602930544001305C400EFD05FF0B3
:1086C00003455401631805061387019E8327C700DD
:1086D00093F737002320F9008327C70093D727009B
:1086E000032707011317E701B3E7E70023A0F4000E
:1086F0002390019E130530008320C10103248101D2
:1087000083244101032901018329C10013010102CE
:10871000678000001385019E2322F500230AF500DF
:1087200013065000930545001305C500EFD05FF018
:108730006FF0DFF4EFD05FFD6FF01FF92390019E23
:108740001305300067800000130101FF232611008C
:10875000239C019EEFF09FC58320C10013010101FE
:1087600067800000130101FF23261100EFF09FC670
:108770008320C1001301010167800000130101FF84
:1087800023261100232481002322910093840500D5
:108790001304060083D7819F130770046380E70AE0
:1087A0006376F7041307A004638EE70E1307200512
:1087B0006390E702EFF0DFCC9307100063FAA71293
:1087C000630804009387819F83A7C7002320F400D8
:1087D000239C019E130530008320C10003248100E7
:1087E000832441001301010167800000638A0708A8
:1087F00013071004E39EE7FC9385819F1386C50051
:1088000093858500EFF05FE09307100063F6A70CF7
:108810009387819F23A207009387819F03A7470027
:108820009307500063E2E7049387819F23A4070026
:1088300023A60700130770042390E7009385819F08
:108840001386C5009385850013050000EFF0DFDB7C
:108850009307100063F6A7089387819F03A7C700BB
:1088600093073000630CF7029387819F83A7C700AB
:10887000638C070413072005239CE19E6FF09FF390
:108880009387819F23A407001307100023A6E70006
:10889000130710042390E7006FF01FF61307A004DE
:1088A000239CE19E13050002EFF0DFC69307100042
:1088B00063FCA7029387819F03A747001307170054
:1088C00023A2E7006FF05FF59387819F83A787005E
:1088D00023A0F4006FF0DFEE130500006FF0DFEF70
:1088E000130500006FF05FEF130500006FF0DFEE7F
:1088F000130500006FF05FEE130101FF2326110046
:10890000232481001304060083D7819F1307600688
:108910006384E7066374F7041307B0066384E7080B
:108920001307F0066390E702EFF09FB5930710007E
:1089300063FCA70A630804009387819F83A7C7008D
:108940002320F400239C019E130530008320C100E6
:10895000032481001301010167800000E39407FEF6
:108960009387819F23A4B7001307200023A6E70065
:10897000130760062390E7009385819F1386C50047
:1089800093858500EFF05FC89307100063F6A70496
:108990009387819F23A4070023A607001307B0062F
:1089A0002390E7009385819F1386C50093858500FA
:1089B00013050000EFF05FC59307100063F2A702F4
:1089C0009387819F83A7C700E38607F61307F00606
:1089D000239CE19E6FF05FF5130500006FF01FF719
:1089E000130500006FF09FF6130500006FF01FF6EF
:1089F00083D781A01307D0046360F72C130101FF14
:108A00002326110023248100232291002320210109
:108A100093040600138905001304050093972700AB
:108A200037270008130787AAB387E70083A7070043
:108A300067800700938781A03707674513073712C0
:108A400023A2E700130780032390E70013064000EA
:108A5000B725024093854500138581A01305450085
:108A6000EFE05FE89307100063FCA720938781A0E5
:108A70003797EFCD1307B79A23A2E7001307A00398
:108A80002390E70013064000B72502409385450078
:108A9000138581A013054500EFE0DFE49307100084
:108AA00063F4A71E1307D0032394E1A0130640002C
:108AB000B725024093850501138581A01305450064
:108AC000EFE0DFC89307100063F4A71C938781A031
:108AD00083A7470093F70708639E070E938781A03B
:108AE00023A487003305240123A6A700938781A030
:108AF00003A7870083A7C7006372F716938781A037
:108B00001307200023A2E700130770042390E70057
:108B100013064000B725024093850501138581A007
:108B200013054500EFE01FDC9307100063F6A7165E
:108B3000130780042394E1A013064000B7250240E8
:108B400093854501138581A013058500EFE09FD92A
:108B50009307100063F6A714938781A003A747002B
:108B60001367070423A2E7001307A0042390E7007C
:108B700013064000B725024093850501138581A0A7
:108B800013054500EFE01FD69307100063FEA71002
:108B9000938781A023A80700938781A003A70701DB
:108BA0009307703E63D2E704938781A083A74700B1
:108BB00013F717006310070893F707016396070878
:108BC000938781A003A787001307074023A4E7002A
:108BD0006FF0DFF19307100023A0F400239401A0AD
:108BE000130520006F0040081307D0042394E1A070
:108BF00013064000B72502409385C500138581A068
:108C000013054500EFE09FB49307100063F2A70A35
:108C1000938781A083A7470093F71700E38607F89F
:108C2000938781A003A707011307170023A8E70074
:108C30006FF09FF69307200023A0F400239401A077
:108C4000130520006F0040029307300023A0F400BA
:108C5000239401A0130520006F00000123A004004D
:108C6000239401A0130530008320C1000324810058
:108C700083244100032901001301010167800000E2
:108C8000130500006FF05FFE130500006FF0DFFDBD
:108C9000130500006FF05FFD130500006FF0DFFCAF
:108CA000130500006FF05FFC130500006FF0DFFBA1
:108CB000130500006FF05FFB239401A01305300043
:108CC00067800000130101FE232E1100232C810078
:108CD000232A91002328210123263101930905002D
:108CE00013840500130906009384060083D781A02E
:108CF00013077006638AE706637CF7041307C00650
:108D0000638CE70A13070007639AE7141306400011
:108D1000B72502409385C500138581A01305450042
:108D2000EFE0DFA29307100063F4A716938781A0FA
:108D300083A7470093F717006380070C938781A0F0
:108D400003A747011307170023AAE7006F00C00914
:108D500063960710938781A01307100023A2E700F2
:108D6000130770062390E70013064000B725024062
:108D700093850501138581A013054500EFE09FB69B
:108D80009307100063FEA70E938781A023A43701E9
:108D900023A80700938781A083A7070163FE870AA2
:108DA000B307F90003A70700938781A023A2E70078
:108DB0001307C0062390E700138581A01306400027
:108DC0008325850013054500EFE0DFB19307100010
:108DD00063FCA70A938781A003A7870013074700B6
:108DE00023A4E70023AA0700938781A003A74701D4
:108DF0009307703E63D8E702938781A083A747005B
:108E000013F717006316070293F74700639C0702E6
:108E1000938781A003A707011307470023A8E70052
:108E20006FF05FF7130700072394E1A06FF01FEEC8
:108E30009307200023A0F400239401A01305200031
:108E40006F0040029307300023A0F400239401A098
:108E5000130520006F00000123A00400239401A04B
:108E6000130530008320C1010324810183244101C3
:108E7000032901018329C100130101026780000059
:108E8000130500006FF01FFE130500006FF09FFD3B
:108E9000130500006FF01FFD83D781A0638C0700CE
:108EA0001307A0086382E702239401A01305300092
:108EB00067800000938781A01307000823A2E700C2
:108EC0001307A0082390E700130101FF23261100D8
:108ED00013064000B725024093850501138581A044
:108EE00013054500EFE01FA09307100063FCA700E7
:108EF000239401A0130530008320C1001301010158
:108F000067800000130500006FF01FFF3725000881
:108F1000130505BE678000001305B00F67800000D1
:108F2000930700001307000063FCB700B306F500C9
:108F300083C606003307D700938717006FF0DFFE64
:108F40001375F70F67800000938701A223A0070025
:108F50001307F0FF23A4E70023A6E70023A80700D8
:108F6000238A0700938701E4130710002380E7009A
:108F7000A380070023A20700678000006F000003A2
:108F8000138701A23307F7008346570113074002F6
:108F9000639EE602138701A22324F7006F000003FB
:108FA00093871700138701A22328F700138701A2D4
:108FB000832707010327070063F2E704138701A251
:108FC000832687001307F0FFE38CE6FA138701A2DC
:108FD0008326C7001307F0FFE394E6FC138701A282
:108FE0003307F7008346570113073002E39AE6FA86
:108FF000138701A22326F7006FF09FFA938701A23F
:1090000083A7870063C80700938601A283A6C600D2
:10901000634CD00293071000631CF704938701A2EE
:1090200003C75701930730006318F704138501A2A3
:1090300093071000230AF500930710002322F50080
:109040001305550167800000138501A21307100066
:10905000230AE500B386F6409386F6FF2322D50067
:10906000938717013305F50013055500678000004D
:1090700013050000678000001305000067800000F2
:10908000938701A203A5470067800000938701A290
:10909000238A070023A0070023A207001307F0FF7D
:1090A00023A4E70023A6E70023A8070067800000A9
:1090B000938701A283C74701639A070683A601A28B
:1090C000130780403307D7406376B7001385070046
:1090D00067800000130101FF232611002324810073
:1090E000232291001384050093050500938401A2B7
:1090F00093860601B386D400130604001385560038
:10910000EF10901583A50400B385850023A0B4005B
:1091100093071000138507008320C10003248100FA
:1091200083244100130101016780000093070000C0
:109130006FF0DFF983C701E463880700138501E45A
:109140001305E5006780000013050000678000003C
:10915000938701E42380070023A2A70093F715005B
:1091600063880702938701E413074002A386E700A0
:1091700083C7170063940702938701E41307B002C3
:109180002386E70023A407001307250023A2E70096
:1091900093F525006390050267800000938701E442
:1091A0001307100023A4E7001307150023A2E7000C
:1091B0006FF01FFE130101FF2326110023248100FD
:1091C000232291002320210193050500138401E44B
:1091D0000329440083248400B3079900B307F400F3
:1091E000130730022386E700130919002322240104
:1091F0001305E400EFF0DFD2B3842401B30494003C
:1092000093060500372600081306C6CD93053000E7
:109210001385C400EF10901F832744009387270015
:109220002322F4008320C100032481008324410011
:1092300003290100130101016780000083C701E4D5
:1092400063900702938701E403A747002320E5000A
:1092500003A587003385A7001305C50067800000BC
:109260001305000067800000938701E423A2070034
:10927000130710002380E70067800000938701E454
:10928000A380A70067800000930600006F004002E3
:10929000130777052380E5006F0080039387770528
:1092A000A380F5009385250013051500938616000D
:1092B00063FAC6028347050013D7470093F7F70008
:1092C00013089000E366E8FC130707032380E5001A
:1092D00013079000E364F7FC93870703A380F5006E
:1092E0006FF05FFC67800000130101FE232E110068
:1092F0002306A10093578500A306F10093570501AB
:109300002307F10013558501A307A10013064000B0
:109310001305C100EFF05FF78320C10113010102C3
:1093200067800000930600006F00000413086004CB
:10933000636EF804938797FC93F7F70F3307E50004
:1093400003471700130890036368E804130707FD39
:109350001377F70F939747003388D500B3E7E700FB
:109360002300F8009386160063F8C60413971600CE
:10937000B307E50083C7070013089003E368F8FA12
:10938000938707FD93F7F70F6FF05FFB938797FACB
:1093900093F7F70F6FF09FFA130860046368E80013
:1093A000130797FC1377F70F6FF0DFFA130797FA9D
:1093B0001377F70F6FF01FFA678000009308000023
:1093C00093070000930600006F0040013388D5002A
:1093D0002300E800938616009387170063FAC702FC
:1093E0003307F500034707001308D007630E070192
:1093F000E38E08FC3388D500134707022300E800FA
:10940000930800006FF01FFD930810006FF0DFFC61
:109410001385060067800000130101FF2326110059
:109420009305300013050000EFF09FD28320C100A8
:109430001301010167800000130101FF23261100C1
:1094400013060040B725000893850506938741253C
:1094500003A50701EF10D017930530001305200076
:10946000EFF01FCF8320C1001301010167800000CE
:109470009387412583D72700638A07009387412577
:10948000239107001305300067800000130101FFDE
:1094900023261100938741253797000813070747B4
:1094A00023AEE70013060040B72500089385450169
:1094B00003A50701EF10D01193053000130530000C
:1094C000EFF01FC993874125239107001305300052
:1094D0008320C1001301010167800000130101FF17
:1094E00023261100232481001384412593060500BF
:1094F000372600081306860593050040032504015E
:10950000EF10C07003250401EF1010079305300021
:10951000EFF01FC48320C100032481001301010167
:10952000678000009387412523900700239107005F
:1095300023920700238C0700A38C0700678000009C
:10954000130101FE232E11009387412503A58700F7
:10955000930681001306C100B7250008938505F91D
:109560001305F501EF10C075032781009307004034
:1095700063F4E7002324F100EFD08FA08327C1001C
:109580003305F5408327810063EAA7042324A10063
:109590009387412583A707011307C0062380E700AF
:1095A000EFD04F9D9387412583A7070103268100B4
:1095B0008325C100B305B50013851700EF105001D6
:1095C000930530000325810013051500EFF05FB807
:1095D0008320C101130101026780000093874125A8
:1095E00083A707011307D0062380E7006FF05FFB16
:1095F000130101FE232E11009387412503A5870047
:10960000930681001306C100B7250008938505F96C
:1096100013057501EF10C06A03278100930700400E
:1096200063F4E7002324F100EFF01F8F8327C100CC
:109630003305F5408327810063EAA7042324A100B2
:109640009387412583A707011307C0062380E700FE
:10965000EFF0DF8B9387412583A707010326810065
:109660008325C100B305B50013851700EF104076C0
:10967000930530000325810013051500EFF05FAD61
:109680008320C101130101026780000093874125F7
:1096900083A707011307D0062380E7006FF05FFB65
:1096A000130101FD232611022324810223229102AA
:1096B000B727000883A847FF938747FF03A8470001
:1096C00003A5870083A5C70003A6070183A647015A
:1096D00003A7870123201101232201012324A100D4
:1096E0002326B1002328C100232AD100232CE10026
:1096F00083D7C701231EF1009387412583D74700F5
:109700006386070213071012638EE70693874125CD
:1097100023920700130530008320C1020324810235
:109720008324410213010103678000001384412553
:109730000326C4001306A6FF135616002326C402F0
:109740000325840093040403938504001305650036
:10975000EFF05FBD8327C4023304F4002308040242
:1097600013065000B7250008938545FE13850400B5
:10977000EF1040626316050293874125130710120C
:109780002392E700EFE08FB29307100063E6A70093
:10979000130500006FF05FF8EFF01FCA6FF01FF7BE
:1097A00013064000B72500089385C5FE13854125A3
:1097B00013050503EF10005E63160500EFF0DFC729
:1097C0006FF0DFF41306D0019387412583A50701CD
:1097D00013050100EFF05FAB930530001305A00304
:1097E000EFF01F976FF09FF29387412583D72700F3
:1097F000639A0704130101FF232611001306F000EA
:10980000B72500089385C5F79387412503A58700F1
:10981000EF10405863140502EFF01FC2130510004B
:10982000EFF0DFA593874125239107001305300052
:109830008320C1001301010167800000EFF0DFBD4C
:109840006FF05FFE938741252391070013053000D9
:10985000678000009387412583D72700639E070C0C
:10986000130101FE232E1100232C81009387412533
:1098700003A5870003441500930770066302F402F2
:1098800093077004630EF4009307D006630AF40094
:109890009307D0046306F40093073006631AF408B4
:1098A0001306C100B7250008938585F71305250029
:1098B000EF100041EFF05FB80317C1009307700687
:1098C0006304F402930770046302F4049307D00660
:1098D0006304F4049307D0046306F40493874125DA
:1098E0002396E74C6F00C000938741252392E74CF5
:1098F0009387412523910700130530008320C10180
:109900000324810113010102678000009387412530
:109910002393E74C6FF0DFFD938741252394E74CB9
:109920006FF01FFD938741252395E74C6FF05FFC97
:10993000EFF09FAE6FF0DFFB938741252391070087
:1099400013053000678000009387412583D72700E7
:10995000638E0700130710186380E7029387412581
:10996000239107001305300067800000938741258D
:10997000130710182391E700130101FF232611009C
:10998000232481001385412513058543EFD01FB89B
:109990009307100063F2A706130400009307000268
:1099A00063C887029387412583A507019316340076
:1099B0001307C41013172700B387E700B385D5003A
:1099C00003A58700EFF05F92130414006FF01FFDF2
:1099D0009305300013058010EFF08FF79387412532
:1099E00023910700130530008320C1000324810068
:1099F0001301010167800000130500006FF0DFFE16
:109A0000130101FF232611002324810093874125A0
:109A100083D7270063840702130770196382E70462
:109A20009387412523910700130530008320C1004F
:109A30000324810013010101678000001384412584
:109A4000032584001306044CB7250008938585F789
:109A500013051500EF10C026930770192311F400A9
:109A6000138541258325054C1305C54BEFD0DFB683
:109A70009307100063E6A700130500006FF01FFBBB
:109A80009387412583A5070103A5C74BEFF0DF8529
:109A90009305300013058000EFF08FEB6FF05FF857
:109AA000130101FE232E1100232C8100232A910093
:109AB00023282101232631019387412583D72700BD
:109AC000638A07021307801B6388E7089387412591
:109AD00023910700130530008320C1010324810175
:109AE00083244101032901018329C10013010102DB
:109AF000678000001384412583248400938414002C
:109B00009305C00213850400EF108024930915000B
:109B10001306840237290008930589F7138504008A
:109B2000EF10001A1306C402930589F71385090084
:109B3000EF1000190327C4029307004063F8E70001
:109B4000938741251307004023A6E7029387412509
:109B50001307801B2391E700138541250326C502C7
:109B60008325850213050503EFD05FBE9307100020
:109B700063E6A700130500006FF01FF6138441256C
:109B80000326C4028325040113050403EFF0CFEF7D
:109B90000325C4029305300013151500EFF04FDBC9
:109BA0006FF0DFF29387412583D72700638E07008C
:109BB0001307A01D6380E7029387412523910700C7
:109BC0001305300067800000938741251307A01D0F
:109BD0002391E700130101FF23261100EFE04F9BC3
:109BE0009307100063F4A702938741251307100021
:109BF000238CE7009387412523910700130530004C
:109C00008320C100130101016780000013050000DB
:109C10006FF01FFF9387412583D72700638E0700CE
:109C20001307901E6380E702938741252391070065
:109C30001305300067800000938741251307901EAD
:109C40002391E700130101FF23261100EFE0CFA6C7
:109C50009307100063F4A7029387412513071000B0
:109C6000238CE700938741252391070013053000DB
:109C70008320C1001301010167800000130500006B
:109C80006FF01FFF130101FE232E1100232C810012
:109C90009387412583D72700638407021307102089
:109CA0006380E70693874125239107001305300061
:109CB0008320C10103248101130101026780000098
:109CC0001384412513074100930681001306C10048
:109CD000B72500089385450403258400EF00507ED6
:109CE0008327C1002328F44C83278100232AF44CC6
:109CF00083274100232CF44C930710202311F400F8
:109D0000938741259386C74D03A6874D83A5474D6D
:109D100003A5074DEFE08FD49307100063F0A7026F
:109D20009387412503A5C74D63160500EFF0CFF0DB
:109D30006FF05FF7EFF08FFA6FF0DFF613050000BA
:109D40006FF01FF7130101FE232E1100232C810059
:109D50009387412583D72700638407021307D02107
:109D60006380E706938741252391070013053000A0
:109D70008320C101032481011301010267800000D7
:109D80001384412513074100930681001306C10087
:109D9000B72500089385C5F803258400EF005072AD
:109DA0008327C1002328F44C83278100232AF44C05
:109DB00083274100232CF44C9307D0212311F40076
:109DC000938741259386C74D03A6874D83A5474DAD
:109DD00003A5074DEFE0CFA09307100063F0A702A3
:109DE0009387412503A5C74D63160500EFF0CFE427
:109DF0006FF05FF7EFF08FEE6FF0DFF61305000006
:109E00006FF01FF79387412583D72700638E0700E4
:109E10001307F0226380E70293874125239107000F
:109E20001305300067800000938741251307F02257
:109E30002391E700130101FF23261100EFD09FE1DA
:109E40009307100063FEA700938741252391070025
:109E5000130530008320C100130101016780000059
:109E6000130500006FF01FFF130101FE232E1100E8
:109E7000232C81009387412583D747006384070201
:109E800013079025638CE7049387412523920700ED
:109E9000130530008320C101032481011301010255
:109EA0006780000013844125032584009306810008
:109EB0001306C100B7250008938505F91305C500F1
:109EC000EF0010608327C1002324F4028327810060
:109ED0002326F402930790252312F400938741254B
:109EE0001386074383A5C70203A58702EFE05FB08F
:109EF0009307100063F0A7029387412503A507434A
:109F000063160500EFF04FD36FF01FF8EFF00FDD91
:109F10006FF09FF7130500006FF0DFF7130101FEEC
:109F2000232E1100232C8100232A910093874125A1
:109F300083D74700638607021307A027638EE706CF
:109F40009387412523920700130530008320C10128
:109F50000324810183244101130101026780000071
:109F600013844125032584001306C100B72500088A
:109F7000938585F71305C500EF0090548327C10032
:109F80002324F402832484009305A0031385C400D2
:109F9000EF00105C130515000326C400B384A44031
:109FA0003306960093050403EFF04FC12326A40265
:109FB0009307A0272312F400938741259386074334
:109FC0001386070383A5C70203A58702EFE09FCF8F
:109FD0009307100063F0A7029387412503A5074369
:109FE00063160500EFF04FC56FF09FF5EFF00FCF50
:109FF0006FF01FF5130500006FF05FF593874125A3
:10A0000083D74700638E07001307D0286380E702D9
:10A0100093874125239207001305300067800000D5
:10A02000938741251307D0282392E700130101FFEE
:10A0300023261100EFE05FE69307100063EAA70014
:10A04000130500008320C100130101016780000097
:10A05000EFF08FBE93874125239207001305300050
:10A060006FF05FFE130101FF2326110023248100FE
:10A070009387412583D727001307E023638EE704E6
:10A080006374F70213070024638EE7081307202484
:10A09000639AE704EFF09FF69307100063E4A704C8
:10A0A000130500006F00C004639E070293874125DB
:10A0B00003A487001306C000B72500089385850117
:10A0C00013050400EF00104D631C05029387412522
:10A0D0001307E0232391E700EFF01FD99307100047
:10A0E00063F4A708938741252391070013053000E7
:10A0F0008320C10003248100130101016780000057
:10A100001306C000B72500089385850213050400D7
:10A11000EF0050486312050293874125130700247E
:10A120002391E700EFF09FDF93071000E3ECA7FA1D
:10A13000130500006FF0DFFB1306A000B725000831
:10A140009385850313050400EF00D044631A0500CE
:10A1500093874125130720242391E7006FF09FF395
:10A16000EFF08FAB6FF01FF8130500006FF05FF892
:10A17000130101FF23261100232481009387412529
:10A1800083D74700638407021307102B6382E70419
:10A190009387412523920700130530008320C100D7
:10A1A00003248100130101016780000013051000E2
:10A1B000EFB05FCF13844125230C040093071000F8
:10A1C000A30CF400EFD0CFA59307102B2312F400BB
:10A1D000EFD05FA893071000E3ECA7FA1305000087
:10A1E0006FF0DFFB130101FF232611002324810000
:10A1F0009387412583D727001307500C6382E70E0E
:10A200001307B00C638CE70863800702938741252E
:10A2100023910700130530008320C100032481002F
:10A2200013010101678000009387412503A4870083
:10A230001306B000B7250008938585F913050400BF
:10A24000EF005035630605061306F001B725000838
:10A25000938545FA13050400EF00D033630C05081D
:10A2600013067001B7250008938545FC130504000B
:10A27000EF0050326304050813066000B72500089C
:10A280009385C5FD13050400EF00D030631C05065F
:10A29000938741251307B00C2391E700EFF04FC0DF
:10A2A00093071000E3E4A7F6130500006FF0DFF654
:10A2B000EFE0DFFC1384412513060040B7250008BA
:10A2C0009385450603250401EF0090309305300087
:10A2D0001305B004EFE0DFE79307500C2311F400FF
:10A2E000EFF01FE993071000E3E2A7F21305000067
:10A2F0006FF09FF2EFF0CFA46FF05FF1EFF04FAF90
:10A300006FF0DFF0EFF04F916FF05FF09387412532
:10A3100083D74700638E07001307B02B6380E702E3
:10A3200093874125239207001305300067800000C2
:10A33000938741251307B02B2392E700130101FFF8
:10A3400023261100EFD0DFA49307100063EAA700D3
:10A35000130500008320C100130101016780000084
:10A36000EFD00F979387412513071000238CE70048
:10A37000A38C070013050000EFB0DFB293874125DF
:10A3800023920700130530006FF0DFFC130101FF7B
:10A39000232611009387412583D727006382070274
:10A3A0001307B01C6386E7029387412523910700BA
:10A3B000130530008320C1001301010167800000F4
:10A3C000EFF08F87938741251307B01C2391E70097
:10A3D000EFF0DFF393071000E3E8A7FC130500009C
:10A3E0006FF05FFD83D741251307400A6360F7389C
:10A3F000130101FF23261100939727003727000838
:10A40000130747CEB387E70083A7070067800700DD
:10A410009387412583C79701639A070C1307400868
:10A42000239AE124EFE09FB59387412523A4A70059
:10A4300063020532EFE0DFC49387412523A6A7001E
:10A44000130770082390E700EFE0DFCE93874125E4
:10A4500023A8A700630405309387412523AA07009A
:10A4600083A7870083C70700130710076380E716D9
:10A47000130710056384E71813078004638EE71839
:10A480001307F0036388E71A130770066382E71C5B
:10A490001307B006638CE71C130730066386E71EBC
:10A4A0001307D0066380E72013070007638AE720BD
:10A4B000130730076384E7221307A007638EE722A0
:10A4C0001307A0056388E724130760076392E72654
:10A4D0001307400A239AE124EFF0DFB89307100036
:10A4E00063E0A710130500006F00801093874125DB
:10A4F00083C78701E38407F2EFE05FA893874125D4
:10A5000023A4A70063040506EFE09FB793874125C6
:10A5100023A6A70083A7870003C70700930730007F
:10A520006314F704930710006310F5041307300752
:10A53000239AE124EFF01F8D9307100063F4A72006
:10A5400093874125238C070013060040B725000898
:10A550009385050503A50701EF00900793053000DB
:10A5600013053000EFE0DFBEEFE05FB293874125D7
:10A5700083C78701638807061307C007239AE1246E
:10A580001385412513054502EFD08FF7930710007F
:10A5900063FEA71A9387412583A7470263840704B4
:10A5A00093874125238C070013060040B725000838
:10A5B0009385450503A50701EF0090019305300041
:10A5C00013053000EFE0DFB86F00C0011307C008CB
:10A5D000239AE124EFF01FC19307100063F4A7183A
:10A5E000EFE0DFAA1307C006239AE1241305100049
:10A5F0008320C10013010101678000001307E008F8
:10A60000239AE124EFF04F9E93071000E3EAA7FCA2
:10A61000130500006FF0DFFD13070009239AE12402
:10A62000EFF04FA393071000E3ECA7FA1305000027
:10A630006FF01FFC13072009239AE124EFE05FE38A
:10A6400093071000E3EEA7F8130500006FF05FFA20
:10A6500013074009239AE124EFF00FAF930710008E
:10A66000E3E0A7F8130500006FF09FF813076009F7
:10A67000239AE124EFF09FD193071000E3E2A7F6BD
:10A68000130500006FF0DFF613078009239AE12419
:10A69000EFF04FD193071000E3E4A7F41305000097
:10A6A0006FF01FF51307A009239AE124EFF04FBFC5
:10A6B00093071000E3E6A7F2130500006FF05FF3C5
:10A6C0001307C009239AE124EFF08FB3930710001A
:10A6D000E3E8A7F0130500006FF09FF11307E0090E
:10A6E000239AE124EFF00FD393071000E3EAA7EEDB
:10A6F000130500006FF0DFEF1307000A239AE1242F
:10A70000EFF04FD893071000E3ECA7EC130500001F
:10A710006FF01FEE1307200A239AE124EFF08FE277
:10A7200093071000E3EEA7EA130500006FF05FEC5B
:10A73000EFE09FCE6FF0DFEA239A0124130530008B
:10A740006FF01FEB130500006FF09FEA1305000088
:10A750006FF01FEA130500006FF09FE9130500007A
:10A760006FF01FE9130500006FF09FE8239A0124A2
:10A770001305300067800000130101FF232611003C
:10A78000EFB0CFEBEFB0CFCBEFE00FFCEFE09FD916
:10A79000EFB00FD0EFB0CFDBEFF0DFC46FF05FFFB3
:10A7A00000000000000000000000000000000000A9
:10A7B0000000000000000000000000000000000099
:10A7C000130101FB23201100232241002324510007
:10A7D0002326610023287100232AA100232CB10025
:10A7E000232EC1002320D1022322E1022324F102DF
:10A7F0002326010323281103232AC103232CD10379
:10A80000232EE1032320F105F322103423205104E9
:10A81000F322003023225104F322407C23245104EC
:10A820007325203493050100EF705FA88322010493
:10A830007390123483224104739002308322810486
:10A840007390427C83200100032241008322810017
:10A850000323C100832301010325410183258101D5
:10A860000326C101832601020327410283278102B7
:10A870000328C10283280103032E4103832E810391
:10A88000032FC103832F010413010105730020303E
:10A8900000000000000000000000000000000000B8
:10A8A00000000000000000000000000000000000A8
:10A8B0000000000000000000000000000000000098
:10A8C000130101FB23201100232241002324510006
:10A8D0002326610023287100232AA100232CB10024
:10A8E000232EC1002320D1022322E1022324F102DE
:10A8F0002326010323281103232AC103232CD10378
:10A90000232EE1032320F10573D0E87E7350F97EF6
:10A9100073D0B97EF390D07E737004308322C1046B
:10A920007390427C83228104739012348322410409
:10A93000739022348320010003224100832281008E
:10A940000323C100832301010325410183258101E4
:10A950000326C101832601020327410283278102C6
:10A960000328C10283280103032E4103832E8103A0
:10A97000032FC103832F010413010105730020304D
:10A98000130605001305000093F615006384060006
:10A990003305C50093D5150013161600E39605FE82
:10A9A000678000006340050663C605061386050040
:10A9B000930505001305F0FF630C060293061000D3
:10A9C000637AB6006358C0001316160093961600FB
:10A9D000E36AB6FE1305000063E6C500B385C54013
:10A9E0003365D50093D6160013561600E39606FE7F
:10A9F0006780000093820000EFF05FFB1385050085
:10AA0000678002003305A04063D80500B305B0405D
:10AA10006FF0DFF9B305B04093820000EFF01FF94B
:10AA20003305A040678002009382000063CA0500DE
:10AA3000634C0500EFF09FF7138505006780020067
:10AA4000B305B040E35805FE3305A040EFF01FF614
:10AA50003305B04067800200B3C7A50093F7370005
:10AA60003307C500639607009307300063E2C7020F
:10AA700093070500637CE50A83C6050093871700EA
:10AA800093851500A38FD7FEE3E8E7FE67800000FB
:10AA90009376350093070500638E060083C6050094
:10AAA0009387170093851500A38FD7FE93F6370081
:10AAB0006FF09FFE9376C7FF138606FE63F4C7060A
:10AAC00083A3050083A2450083AF850003AFC500C3
:10AAD00083AE050103AE450103A3850183A8C5012B
:10AAE0009385450223A0770003A8C5FF23A2570042
:10AAF00023A4F70123A6E70123A8D70123AAC701AE
:10AB000023AC670023AE17019387470223AE07FFEC
:10AB10006FF0DFFA03A60500938747009385450091
:10AB200023AEC7FEE3E8D7FEE3E8E7F46780000062
:10AB30001303F00013070500637EC3029377F70049
:10AB40006390070A63920508937606FF1376F60072
:10AB5000B386E6002320B7002322B7002324B700E2
:10AB60002326B70013070701E366D7FE6314060028
:10AB700067800000B306C34093962600970200004A
:10AB8000B38656006780C6002307B700A306B70048
:10AB90002306B700A305B7002305B700A304B70039
:10ABA0002304B700A303B7002303B700A302B70031
:10ABB0002302B700A301B7002301B700A300B70029
:10ABC0002300B7006780000093F5F50F939685008A
:10ABD000B3E5D50093960501B3E5D5006FF0DFF638
:10ABE0009396270097020000B386560093820000D8
:10ABF000E78006FA93800200938707FF3307F74048
:10AC00003306F600E378C3F66FF0DFF3130101F6C5
:10AC1000232AF108232A91062326D1082328E108B4
:10AC2000232C0109232E110993874181232E11061C
:10AC3000232C810683A4070063D205029307B00882
:10AC400023A0F4001305F0FF8320C107032481072C
:10AC5000832441071301010A6780000093078020C5
:10AC6000231AF1002324A100232CA1009307000044
:10AC7000638405009387F5FF2328F100232EF1005C
:10AC80009306C1089307F0FF1384050013850400A1
:10AC900093058100231BF1002322D100EF00802DBA
:10ACA0009307F0FF6356F5009307B00823A0F40064
:10ACB000E30C04F883278100238007006FF0DFF89E
:10ACC000130101F52322F10A9307402023261108DE
:10ACD0002326B100232CC108232ED1082320E10A0A
:10ACE0002324010B2326110B2312F102232CA10094
:10ACF0002324A102EF00400897070000938707056F
:10AD0000232EF1029307F0FF8325C1002313F102E4
:10AD100093874181232EA1002326A10203A50700CA
:10AD200093068109138605009305810123260104FA
:10AD300023200106232AD100EF0080748320C1085C
:10AD40001301010B678000001305000067800000FD
:10AD500093F5F50F83470500638A07006394B700F6
:10AD600067800000130515006FF0DFFE63840500A7
:10AD70001305000067800000930705009387170004
:10AD800003C7F7FFE31C07FE3385A7401305F5FF54
:10AD900067800000630A06021306F6FF130700002F
:10ADA000B307E500B386E50083C7070083C6060046
:10ADB0006398D7006306C70013071700E39207FEE6
:10ADC0003385D740678000001305000067800000CE
:10ADD00093070500630E06009385150003C7F5FF72
:10ADE000938717001306F6FFA38FE7FEE31407FE11
:10ADF0003386C7006394C7006780000093871700FD
:10AE0000A38F07FE6FF01FFF130101FE232821010E
:10AE100003A98500232C8100232441012320610103
:10AE2000232E1100232A91002326310123225101D0
:10AE300013840500130B0600138A060063E0260F37
:10AE400083D7C50013F707486308070C8324040061
:10AE50000327440183A50501930A0500B389B44083
:10AE6000931417003387E4009354F701B384E4008C
:10AE70001387160093D414403307370163F4E400BA
:10AE80009304070093F707406384070C938504003D
:10AE900013850A00EF101052130905006312050410
:10AEA0009307C00023A0FA008357C4001305F0FFE6
:10AEB00093E707042316F4008320C10103248101D2
:10AEC00083244101032901018329C100032A810050
:10AED000832A4100032B0100130101026780000057
:10AEE0008325040113860900EFF01FB78357C400C0
:10AEF00093F7F7B793E707082316F40023282401F4
:10AF0000232A940033093901B384344123202401D6
:10AF10002324940013090A0063742A0113090A0008
:10AF2000032504001306090093050B00EF101032EF
:10AF30008327840013050000B38727412324F400EE
:10AF40008327040033892701232024016FF0DFF6D3
:10AF50001386040013850A00EF10905B13090500A7
:10AF6000E31E05F88325040113850A00EF10D03392
:10AF70006FF01FF383D7C500130101F52322910A57
:10AF80002320210B232E31092326110A2324810A91
:10AF9000232C4109232A51092328610923267109F9
:10AFA000232481092322910993F7070893090500B7
:10AFB00013890500930406006388070683A705012B
:10AFC00063940706930500042326D100EF10903EFA
:10AFD0002320A9002328A9008326C10063120504A9
:10AFE0009307C00023A0F9001305F0FF8320C10AD6
:10AFF0000324810A8324410A0329010A8329C10900
:10B00000032A8109832A4109032B0109832BC108E3
:10B01000032C8108832C41081301010B6780000079
:10B0200093070004232AF90093070002A30CF102FE
:10B0300093070003232A0102230DF102232ED100DE
:10B04000130B5002977AFFFF938ACA06930B1000E6
:10B05000175CFFF7130C0CFB1384040083470400F8
:10B06000638407006396670DB30C944063860C02FB
:10B0700093860C00138604009305090013850900CC
:10B08000EFF09FD89307F0FF630EF524832641036A
:10B09000B3869601232AD1028347040063840724E0
:10B0A0009307F0FF930414002320010223260102DA
:10B0B0002322F10223240102A3010106232C01060D
:10B0C00083C504001306500013850A00EF10D01545
:10B0D00013841400832701026310050613F7070188
:10B0E0006306070013070002A301E10613F78700B8
:10B0F000630607001307B002A301E10683C604003C
:10B100001307A0026386E6040327C1021384040028
:10B110009307000013069000834604009305140073
:10B12000938606FD637AD610639E07026F000005C2
:10B13000130414006FF09FF2330555413395AB00B3
:10B14000B3E7A7002320F102930404006FF05FF738
:10B150000327C1019306470003270700232ED100D0
:10B16000634607002326E1026F0040013307E040F9
:10B1700093E727002326E1022320F102034704007E
:10B180009307E0026316F702034714009307A00237
:10B190006316F70C8327C1011304240013874700AB
:10B1A00083A70700232EE10063C6070A2322F102CA
:10B1B00083450400130630001775FFFF130505F0E3
:10B1C000EF109006630405029777FFFF938707EF60
:10B1D0003305F54093070004B397A7000325010248
:10B1E000130414003365F5002320A10283450400F5
:10B1F000130660001775FFFF130585EC9304140018
:10B20000230CB102EF105002630A050E63160C0AFC
:10B21000032701028327C10113770710630607087C
:10B2200093874700232EF10083274103B38747010B
:10B23000232AF1026FF05FE293172700B387E7003C
:10B24000939717003387D7001384050093071000E6
:10B250006FF09FEC9307F0FF6FF05FF5130414009D
:10B260002322010293070000130700001306900039
:10B270008346040093051400938606FD6378D60088
:10B28000E38807F22322E1026FF09FF29317270071
:10B29000B387E700939717003387D700138405001F
:10B2A000930710006FF0DFFC9387770093F787FF19
:10B2B000938787006FF01FF71307C10197060000FF
:10B2C0009386C6B41306090093050102138509008D
:10B2D00097000000E70000009307F0FF130A050045
:10B2E000E314F5F48357C9001305F0FF93F707043F
:10B2F000E39E07CE032541036FF05FCF1307C10123
:10B3000097060000938686B0130609009305010294
:10B3100013850900EF00007E6FF01FFC130101FF91
:10B3200023261100232481002322910023202101C0
:10B330009307F0FF6392F5029304F0FF8320C100AE
:10B3400003248100138504000329010083244100A4
:10B3500013010101678000008357C60013F9F50F40
:10B3600093F4F50F93F7F7FD2316F60083274603B2
:10B37000032746006380070483278603130406001F
:10B380006352F702832704001387F7FF2320E400AA
:10B39000A38F27FF83274400938717002322F400FD
:10B3A0006FF0DFF993050600EF100053E30C05FC86
:10B3B0006FF09FF88326060183270600638206024A
:10B3C00063F0F60283C6F7FF639C96009387F7FF4E
:10B3D000130717002320F6002322E6006FF01FF664
:10B3E000232EF60293074604232AF6029307300021
:10B3F000232CF602930766042320F600930710001F
:10B400002320E604230326052322F6006FF01FF312
:10B41000130101FF232481001384050083A5450344
:10B4200023261100638E0502930744046384F5000C
:10B43000EF10806783270404232A04022322F400E8
:10B44000638007028327C403130500002320F40050
:10B450008320C100032481001301010167800000E3
:10B4600083270401232204001305F0FF2320F400A6
:10B470008357C40093E707022316F4006FF05FFDC3
:10B48000130101D297070000938787E92328212D14
:10B49000232CF1281309C10197070000938787F730
:10B4A000232C812C232A912C2326312D2324412D3A
:10B4B0002322512D2320612D232E712B232C812B10
:10B4C000232E112C232A912B2328A12B2326B12BA9
:10B4D000930405001384050023240112232601127E
:10B4E00023282113232EF128232CD1009309500265
:10B4F000930AA002130B9000177AFFFF130A0ABCED
:10B50000930B7006175CFFF7130CCCAF8347060054
:10B510002326C10063840742EF1040490326C1007F
:10B52000834D0600930C16003305B50183471500C3
:10B5300093F7870063860706832744006356F00469
:10B54000EF10C0468327040003C707003305E5005A
:10B5500003471500137787006316070013860C0056
:10B560006FF0DFFA0327C112938717002320F4003E
:10B57000130717002326E112032744001307F7FFE0
:10B580002322E4006FF05FFB8327C12993050400A9
:10B5900013850400E7800700E30405FA6FF01FFC41
:10B5A00063903D1D23220112232E011083471600B4
:10B5B0006398570193070001232EF110930C260086
:10B5C00083C50C00138D0C00938C1C00938705FD24
:10B5D0006378FB061306300013050A00EF10C04421
:10B5E000630005023305454193071000B397A70098
:10B5F0000325C111138D0C003365F500232EA11016
:10B6000083470D00930C1D0063E6FB1013075006E3
:10B6100063F2E724130770046364F704130750040C
:10B6200063FAE72263880718638C371393073000A7
:10B63000232AF1129307A0002320F1126F00C00506
:10B640000327411293172700B387E700939717004A
:10B65000938707FDB387B7002322F1126FF05FF6DF
:10B660001307B005638CE716636AF70813078005B4
:10B67000E39EE7FA0327C11113670720232EE11089
:10B68000130700012320E1121307E006B337F70088
:10B6900093873700232AF112832744006350F01C5C
:10B6A0008327C11193F7070463900702EF1000305E
:10B6B0008327040003C707003305E500034715008F
:10B6C000137787006318071A832741131307200095
:10B6D0006342F71E93068101130604009305C1110E
:10B6E00013850400EF00C07E930710006308F52463
:10B6F00093072000E314F5E66F00400B13073006B4
:10B700006380E71013074006E392E7F21307A000F7
:10B710006FF05FF7130700076382E70A6362F702BF
:10B720001307E0066388E70E6362F70A13079006C3
:10B73000E39EE7EE23200112930730006FF09FF5A0
:10B7400013075007E384E7FC13078007E384E7F25D
:10B7500013073007E39CE7EC930720006FF09FF39B
:10B7600083274400635AF0028327040003C70700BD
:10B770006316B71D93871700032744002320F400A6
:10B780008327C1121307F7FF2322E40093871700D2
:10B790002326F1126FF09FDC8327C1299305040053
:10B7A00013850400E7800700E30005FC03258112F0
:10B7B000631205141305F0FF6F0080140327C111F5
:10B7C00013670702232EE1106FF0DFEA9307800072
:10B7D0002320F112930740006FF0DFEB93850C00FC
:10B7E00013050900EF00D03F8327C111930C05001A
:10B7F00093E70704232EF110930710006FF09FE9E1
:10B800008327C111232A011293E70704232EF11085
:10B810006FF09FE88327C11113F70701E31007D4E6
:10B820000327810193F517008326C11213064700F1
:10B83000638A0500232CC100832707002390D700CB
:10B840006FF0DFD1232CC1008327070023A0D7008E
:10B850006FF0DFD0930750006FF0DFE38327C1293B
:10B860009305040013850400E7800700E30A05E25E
:10B870006FF0DFF30327C112130717002326E1122D
:10B88000032744001307F7FF2322E4006358E00076
:10B89000938717002320F4006FF05FE18327C1290D
:10B8A0009305040013850400E7800700E30005E02A
:10B8B0006FF0DFEF13074000634EF700930681013E
:10B8C000130604009305C11113850400EF004079AD
:10B8D0006FF09FE1E3040CC8930681011306040096
:10B8E0009305C1111385040097000000E7000000D4
:10B8F0006FF09FDF8357C40093F70704E39C07EAC8
:10B900008320C12D0324812D8324412D0329012D62
:10B910008329C12C032A812C832A412C032B012C3F
:10B92000832BC12B032C812B832C412B032D012B2B
:10B93000832DC12A1301012E678000000325811287
:10B940006FF01FFC130101FD232A510183A705019C
:10B95000930A070003A78500232481022322910272
:10B96000232E3101232C4101232611022320210300
:10B970002328610123267101930905001384050022
:10B9800093040600138A060063D4E70093070700B8
:10B9900023A0F400034734046306070093871700CD
:10B9A00023A0F4008327040093F7070263880700AD
:10B9B00083A704009387270023A0F4000329040031
:10B9C00013796900631E0900130B9401930BF0FFB8
:10B9D0008327C40003A70400B387E7406342F90844
:10B9E000832704008346340493F70702B336D0005C
:10B9F0006390070C1306340493050A0013850900AD
:10BA0000E7800A009307F0FF6308F5068327040028
:10BA10001306400003A7040093F767008326C400C1
:10BA2000930400006398C700B384E64063D4040025
:10BA30009304000083278400032704016356F70062
:10BA4000B387E740B384F400130900001304A40192
:10BA5000130BF0FF63902409130500006F00000230
:10BA60009306100013060B0093050A0013850900C6
:10BA7000E7800A00631A75031305F0FF8320C102F3
:10BA80000324810283244102032901028329C10185
:10BA9000032A8101832A4101032B0101832BC10069
:10BAA0001301010367800000130919006FF05FF2B2
:10BAB0003307D40013060003A301C704034754044B
:10BAC00093871600B307F40093862600A381E7044A
:10BAD0006FF05FF2930610001306040093050A004E
:10BAE00013850900E7800A00E30865F913091900C6
:10BAF0006FF05FF6130101FC232C81022326310332
:10BB00002322510323206103232E7101232E1102CE
:10BB1000232A91022328210323244103232C81017A
:10BB200083C78501938B06009306E006930A050000
:10BB300013840500130B060093893504638CD72802
:10BB400063E8F60693063006638CD70A63ECF600CA
:10BB50006380072C930680056388D712130C240496
:10BB60006F00400B930640066386D700930690064D
:10BB7000E396D7FE832704000326070093F5070802
:10BB800093064600638E0508832406002320D70011
:10BB900063D804009307D002B3049040A301F404D7
:10BBA000176AFFFF130A4A521309A0006F00C01260
:10BBB000930630076384D72663E2F6029306F00605
:10BBC000638ED70693060007E39AD7F883A705008C
:10BBD00093E7070223A0F5006F004001930650078A
:10BBE000638ED70493068007E39AD7F693078007FE
:10BBF000A302F404176AFFFF130A4A4E6F0080097C
:10BC000083270700138C25049386470083A707002A
:10BC10002320D7002301F404930710006F000023B2
:10BC20008324060093F707042320D700E38207F656
:10BC30009394040193D404416FF09FF5032604000C
:10BC400083260700137506089385460063080500E0
:10BC50002320B70083A406006F004001137606047A
:10BC60002320B700E30806FE83D406001307F0067E
:10BC7000176AFFFF130A4A451309A000639CE704F3
:10BC8000130980006F000005A382F504176AFFFF07
:10BC9000130A8A43832704008326070013F6070844
:10BCA00083A4060093864600630606102320D7006F
:10BCB00013F717006306070093E707022320F40039
:10BCC00013090001639804008327040093F7F7FD2C
:10BCD0002320F400A3010404832744002324F40058
:10BCE00063C80700032704001377B7FF2320E4008D
:10BCF00063960400138C0900638A0702138C090001
:10BD00009305090013850400EFE0DFCE3305AA0098
:10BD100083470500130CFCFF930509002300FC007A
:10BD200013850400EFE09FC863F2240B93078000A3
:10BD30006314F9028327040093F71700638E07004A
:10BD4000032744008327040163C8E7009307000327
:10BD5000A30FFCFE130CFCFFB38989412328340197
:10BD600013870B0093060B001306C1009305040014
:10BD700013850A00EFF01FBD9304F0FF631E950CBE
:10BD80001305F0FF8320C1030324810383244103AF
:10BD9000032901038329C102032A8102832A410264
:10BDA000032B0102832BC101032C81011301010428
:10BDB0006780000013F607042320D700E30A06EE8D
:10BDC0009394040193D404016FF09FEE9304050053
:10BDD0006FF01FF383A605008327070003A6450124
:10BDE00013F5060893854700630A05002320B70072
:10BDF00083A7070023A0C7006F0080012320B7009E
:10BE000093F6060483A70700E38606FE2390C70087
:10BE100023280400138C09006FF09FF48327070088
:10BE200003A6450093050000938647002320D70012
:10BE300003AC070013050C00EF00103F630605007C
:10BE4000330585412322A400832744002328F400DE
:10BE5000A30104046FF0DFF08326040113060C0035
:10BE600093050B0013850A00E7800B00E30A95F0A9
:10BE70008327040093F72700639407048327C100F6
:10BE80000325C400E350F5F0138507006FF09FEF22
:10BE9000930610001306090093050B0013850A0092
:10BEA000E7800B00E30E35ED938414008327C40074
:10BEB0000327C100B387E740E3CCF4FC6FF01FFC1D
:10BEC00093040000130994019309F0FF6FF01FFE23
:10BED00083A78500130101FE232C8100232A9100F2
:10BEE00023244101232E110023282101232631017F
:10BEF0002322510123206101130A05001384050048
:10BF000093040600639C070003A7850193071000B4
:10BF1000630407009307F0FF2324F4008327040041
:10BF200093F70701639A070083A70600138747006A
:10BF300023A0E60083A9070013090000930A10005C
:10BF4000130B200003258401630605046310550FBD
:10BF500083A7040003C7070083274401B387E700D2
:10BF600083C7070063980702631609088320C1018D
:10BF70000324810183244101032901018329C10094
:10BF8000032A8100832A4100032B010013010102CF
:10BF900067800000832704001309190093F7070145
:10BFA000639A070083A704009389190083C70700D9
:10BFB000A38FF9FE03A7040083A74400130717000B
:10BFC00023A0E400032784009387F7FF23A2F40053
:10BFD0001307F7FF2324E400630E0700E344F0F6A1
:10BFE000832704189385040013050A00E7800700DF
:10BFF000E30A05F48327040093F70701639E070013
:10C000008327C400938717002326F4008327840125
:10C0100063840700238009008327040113050000BF
:10C0200033892701232824016FF05FF4631065032F
:10C03000EF00D01783A7040083C707003305F5007E
:10C040008347150093F78700E38607F4E31409FAA2
:10C050000325840193071000E31EF5F86FF01FF12C
:10C06000130101FB9767FFFF9387C7092320210571
:10C070002322F100138906009767FFFF9387C70803
:10C0800083A685012324F1009767FFFF93870708A4
:10C0900023248104232E310323286103232EB1019D
:10C0A0002326F1002326110423229104232C41038B
:10C0B000232A51032326710323248103232291037E
:10C0C0002320A10393073000930905001384050082
:10C0D000930D0600170B0000130B8B7E6396F60082
:10C0E000170B0000130B4B5C832784009306C015CD
:10C0F000130A00001386F7FF63F8C600138A37EAB5
:10C100009307D0152324F40083270400B7160000FA
:10C11000938606D09304C401B3E7D7002320F4002C
:10C12000130C4100938A0400930B0000930C002031
:10C1300083A70D0003250C001306200083C507000C
:10C14000EF00900E63020508930710006390FB1444
:10C1500083274400639C07008327040013078000A3
:10C160002322E40093E707202320F4008327040020
:10C1700093F7F7AF2320F400832784001386F7FF9B
:10C180002324C4006382070403A60D00138D1A0044
:10C190009307160023A0FD00034606002380CA0073
:10C1A00003A64D00930A0D001306F6FF23A2CD004F
:10C1B000634CC0000326041893850D001385090005
:10C1C000E7000600631A0518938B1B0093073000E5
:10C1D000130C4C00E39EFBF4832744006396070096
:10C1E0009307A0002322F400832744000325440181
:10C1F0009765FFFF9385C5F0B385F540B7FBFFFF5B
:10C20000371C0000138D0A00EF00801D930A000008
:10C21000930C0003938BFB6F130C0C80832684001C
:10C2200003260400638C060A03A50D008325440140
:10C2300003480500B385050183C505006380050A31
:10C2400063189807B375860163840506938A1A00FC
:10C2500063080A0093861600130AFAFF2324D40009
:10C2600083A64D009386F6FF23A2DD00635ED00413
:10C2700083A60D009386160023A0DD00832684008C
:10C280009386F6FF2324D4006FF05FF99307200014
:10C29000E394FBEE8327040013F60760E31696F39E
:10C2A000130700012322E40093E707106FF09FECCF
:10C2B000337676012320C40083460500130D1D004C
:10C2C000A30FDDFE6FF0DFF98326041893850D00C0
:10C2D00013850900E7800600E30205FA83260400BF
:10C2E00093F606106386060263F0A4038345FDFF00
:10C2F0008326C417130AFDFF13860D00138509005A
:10C30000E7800600130D0A001305100063089D085E
:10C3100003270400137707016316070623000D00A7
:10C32000832644001306000093850400138509004A
:10C33000E7000B00832604000327090013F606021A
:10C3400063000602930647002320D9000327070055
:10C350002320A7006F004002930A00006FF01FF82F
:10C3600093F5160013064700638805062320C900CD
:10C37000032707002310A7000327C4001307170093
:10C380002326E40083270401B3049D40B3845401B1
:10C39000B384970023289400130500008320C10470
:10C3A0000324810483244104032901048329C10354
:10C3B000032A8103832A4103032B0103832BC10238
:10C3C000032C8102832C4102032D0102832DC10124
:10C3D00013010105678000002320C9006FF01FF7DB
:10C3E00083C705001307E0056380E7061387150080
:10C3F0009306000013060000930500103308C500E3
:10C400002300D80013061600E31AB6FE1306F7FF42
:10C410006388070293C616009308D0021308D0055C
:10C420003306F5002300D6008345070013061700E6
:10C43000638E1503638605016390050213060700EA
:10C4400013050600678000001387250083C71500C9
:10C45000930610006FF01FFA93870500130706007C
:10C460006FF01FFC9307D0026FF05FFF834517004A
:10C47000E38A05FFE3C8F5FE13072700938717003B
:10C480003306F5002300D600E3CAB7FE6FF0DFF9EC
:10C49000130101FB23202105232E3103232C41030B
:10C4A000232A510323286103232611042324810412
:10C4B0002322910423267103232481032322910341
:10C4C0002320A103232EB101130B0500138A0500BD
:10C4D000930A0600138906009389050093841900C6
:10C4E00003C4F4FF130507002326E100EF00804B8F
:10C4F00033058500834715000327C10093F78700A4
:10C500006398070C9307D0026318F40C03C404006B
:10C51000130C100093842900630E09169307000181
:10C520006314F902930700036310F40283C7040045
:10C530001307800593F7F70D6396E71403C41400FF
:10C540001309000193842400B709008063140C00D0
:10C5500093C9F9FF9305090013850900EFE08FC91E
:10C56000930B05009305090013850900EFE00FC444
:10C57000930C05001307000013050000930D9000B5
:10C58000130D90019306F0FF930704FD63E4FD068D
:10C5900013840700635024096306D7021307F0FFD2
:10C5A00063E2AC026394AC0063CE8B00930505009C
:10C5B00013050900EFE0CFBC3305A40013071000FA
:10C5C0009306F0FF9384140003C4F4FF6FF0DFFBC5
:10C5D000938904006FF09FF09307B0026306F400A4
:10C5E000130C00006FF05FF303C404009384290070
:10C5F0006FF01FFF9307F4FB6366FD00130494FCC8
:10C600006FF05FF99307F4F96366FD00130494FA81
:10C610006FF05FF89307F0FF6318F70493072002A9
:10C620002320FB001385090063980A048320C104BA
:10C630000324810483244104032901048329C103C1
:10C64000032A8103832A4103032B0103832BC102A5
:10C65000032C8102832C4102032D0102832DC10191
:10C66000130101056780000063040C003305A0403E
:10C67000E38E0AFA63040700138AF4FF23A04A0139
:10C680006FF0DFFA13040003E31009EC13098000D4
:10C690006FF09FEB93070003E30AF4E81309A0008F
:10C6A0006FF09FEA9387418183A7070003A70702E2
:10C6B000631607001747FF17130787E46FF05FDD66
:10C6C000130101FC232821032326310323244103E2
:10C6D0002322510323206103232E1102232C8102E4
:10C6E000232A9102232E7101232C8101232A9101F7
:10C6F0002328A101930A0500138A0500130B0600E5
:10C7000013890600938905009384190003C4F4FF7C
:10C71000130507002326E100EF00C028330585003C
:10C72000834715000327C10093F78700639E070A1C
:10C730009307D002631EF40A03C404009384290003
:10C740009309100063040916930700016314F902AA
:10C75000930700036310F40283C7040013078005E6
:10C7600093F7F70D639CE71203C41400130900014B
:10C7700093842400930509001305F0FFEFE00FA355
:10C78000930B0500930509001305F0FFEFE08FA65A
:10C79000930C05001307000013050000130D900013
:10C7A000130C9001930704FD6362FD0613840700D8
:10C7B00063522409634C07061307F0FF63E0AB02E2
:10C7C0006394AB0063CC8C0093050500130509004E
:10C7D000EFE00F9B3305A4001307100093841400AF
:10C7E00003C4F4FF6FF01FFC938904006FF0DFF1C6
:10C7F0009307B0026306F400930900006FF09FF402
:10C8000003C40400938429006FF01FFF9307F4FB17
:10C810006366FC00130494FC6FF09FF99307F4F92E
:10C82000636AFC00130494FA6FF09FF81307F0FF9B
:10C830006FF0DFFA635607049307200223A0FA0083
:10C840001305F0FF63160B048320C1030324810347
:10C8500083244103032901038329C102032A81029E
:10C86000832A4102032B0102832BC101032C810186
:10C87000832C4101032D0101130101046780000095
:10C88000638409003305A040E3000BFC6304070048
:10C89000138AF4FF23204B016FF01FFB13040003E6
:10C8A000E31A09EC130980006FF0DFEC9307000333
:10C8B000E304F4EA1309A0006FF0DFEB93874181F2
:10C8C00083A7070003A70702631607001747FF1790
:10C8D000130707C36FF0DFDE130101FE232C810075
:10C8E0001384050083A54503232E1100232A9100FC
:10C8F00023282101232631012324410193074404E5
:10C900006394F50693050040EF00C02A6314050206
:10C910001305F0FF8320C101032481018324410119
:10C92000032901018329C100032A810013010102A7
:10C930006780000093070040232CF40283476404BF
:10C94000232AA4021305D53F2301F500834754048D
:10C95000A300F500834744042300F5002320A4002E
:10C96000130500006FF01FFB0329840393191900BE
:10C9700013860900EF00C03993040500E30A05F8A7
:10C98000330A2501930505001306090013050A0063
:10C99000EFE08F8C23204401232A9402232C3403BC
:10C9A0006FF01FFC0325C50E67800000938741814F
:10C9B00083A7070083A70702639607009747FF171F
:10C9C000938707B403A5C70E67800000639A05022A
:10C9D000130101FF9305C10013050000630E06005B
:10C9E0001305E0FF638A06008347060023A0F500D5
:10C9F000034506003335A0001301010167800000E4
:10CA000013050000630006021305E0FF638C0600B7
:10CA10008347060023A0F500034506003335A00038
:10CA2000678000006780000093F5F50F3306C500AE
:10CA30006316C500130500006780000083470500EA
:10CA4000E38CB7FE130515006FF09FFE63FAA50493
:10CA5000B386C5006376D5049345F6FF93070000BF
:10CA60009387F7FF6394F500678000003387F60033
:10CA7000034807003387C7003307E5002300070199
:10CA80006FF01FFE3387F500834607003307F5007C
:10CA9000938717002300D700E316F6FE6780000097
:10CAA000930700006FF05FFF6384051083A7C5FF45
:10CAB000130101FF2324810023261100232291006A
:10CAC0001384C5FF63D407003304F4009304050006
:10CAD000EF00C0349747FF179387C7BC83A70700B1
:10CAE00063940702232204009747FF1723AC87BAF9
:10CAF000032481008320C1001385040083244100A6
:10CB0000130101016F00C0316376F4028326040033
:10CB10003307D400639AE70003A7070083A7470001
:10CB20003307D7002320E4002322F4006FF0DFFB5B
:10CB30009307070003A7470063040700E37AE4FEB6
:10CB400083A607003386D7006318860203260400F5
:10CB5000B386C60023A0D7003386D700E31AC7F8F0
:10CB60000326070003274700B306D60023A0D700FB
:10CB700023A2E7006FF0DFF76378C4009307C000DB
:10CB800023A0F4006FF0DFF603260400B306C40010
:10CB9000631AD7008326070003274700B386C60021
:10CBA0002320D4002322E40023A287006FF05FF447
:10CBB00067800000130101FE232A91009384350051
:10CBC00093F4C4FF232E1100232C8100232821017C
:10CBD00023263101938484009307C00063FAF4068E
:10CBE0009304C00063E8B40613090500EF000023B6
:10CBF0009747FF17938707AB03A7070013040700A6
:10CC0000631E04069747FF17938707AA83A70700A9
:10CC1000639C07009305000013050900EF00C0188E
:10CC20009747FF1723A2A7A89385040013050900BF
:10CC3000EF0080179309F0FF631C350B9307C000CA
:10CC40002320F90013050900EF00801D6F0000018B
:10CC5000E3DA04F89307C0002320F5001305000071
:10CC60008320C1010324810183244101032901019F
:10CC70008329C1001301010267800000832704009B
:10CC8000B387974063C007069306B00063FAF600C7
:10CC90002320F4003304F400232094006F004001AB
:10CCA00083274400631C87021747FF17232CF79E36
:10CCB00013050900EF00C0161305B40093074400E4
:10CCC000137585FF3307F540E30C07F83304E400E0
:10CCD000B387A7402320F4006FF09FF82322F700CA
:10CCE0006FF01FFD13070400032444006FF05FF191
:10CCF000130435001374C4FFE30085FAB305A440A0
:10CD000013050900EF00400AE31835F96FF01FF32F
:10CD100063960500930506006FF0DFE9130101FE3D
:10CD2000232C8100232E1100232A91002328210186
:10CD3000232631011304060063160602EFF0DFD646
:10CD4000130900008320C101032481011305090098
:10CD500083244101032901018329C1001301010238
:10CD6000678000009384050093090500EF00800BA5
:10CD700013890400E37885FC9305040013850900FA
:10CD8000EFF05FE313090500E30E05FA9385040055
:10CD900013060400EFD05FCC9385040013850900CF
:10CDA000EFF09FD06FF01FFA130101FF23248100E1
:10CDB000130405001385050023A001782326110024
:10CDC000EF50CFD09307F0FF631AF50093870178F7
:10CDD00083A70700638407002320F4008320C10099
:10CDE00003248100130101016780000063840502B0
:10CDF0009307F00F63FAC7009307A0082320F500FC
:10CE00001305F0FF678000002380C50013051000A4
:10CE10006780000013050000678000006780000045
:10CE20006780000083A7C5FF1385C7FF63D807008D
:10CE3000B385A50083A705003305F50067800000D2
:04CE400000000300EB
:08CE4400400080000000000026
:04CE4C0003020102DA
:04CE500004030904CA
:10CE540009024300020100803209040000010202B9
:10CE6400010005240010010524010001042402022C
:10CE740005240600010705820308000A09040100CD
:10CE8400020A0000000705030240000007058102B2
:10CE940040000000FF000000B85900080C5A0008C8
:10CEA4003C5B0008A05A0008505A0008000000002B
:10CEB400000000000000000000000000000000006E
:10CEC400000000000000000000000000000000005E
:10CED400000000000000000000000000000000004E
:10CEE400000000000000000000000000000000003E
:10D2C400000000000000000000000000240300082B
:10D2D40000000020000000003803000800000000E7
:10D2E400000000000000000000000000000000003A
:10D2F4002C2100084C2100080C210008000000002B
:10D304000000000000000000000000000000000019
:10D314000000000000000000000000000000000009
:10D3240000000000000000000000000000000000F9
:10D3340000000000000000000000000000000000E9
:10D344000000000000000000000000004300000096
:10D3540000000000000000000000000000000000C9
:10D364000000000000000000000000004300000076
:10D3740000000000000000000000000000000000A9
:10D384000000000000000000000000004300000056
:10D394000000000000000000000000000000000089
:10D3A4000000000000000000000000004300000036
:10D3B4000000000000000000000000000000000069
:10D3C4000000000000000000000000004300000016
:10D3D4000000000000000000000000000000000049
:10D3E40000000000000000000000000043000000F6
:10D3F4000000000000000000000000000000000029
:10D4040000000000000000000000000043000000D5
:10D414000000000000000000000000000000000008
:10D42400000000000000000000000000ECCD000837
:10D43400CCC90008000000007C2100087821000805
:10D4440024200008242000082420000824200008A8
:10D454002420000824200008242000082420000898
:10D4640024200008FFFFFFFFFFFFFFFFFFFFFFFF78
:10D47400FFFF000001004153434949000000000040
:10D484000000000000000000000000000000000098
:10D49400000000000000415343494900000000001F
:10D4A4000000000000000000000000000000000078
:10D4B4000000000000000000F0150020FF00000044
:10D4C40000C2010000000800010100009C040020CB
:08D4D400000000000102030446
:040000050800015C92
:00000001FF
